:020000020000FC
:02000000EEC050
:02000800567828
:100034000C94072F0C94052F4156522D4368697078
:100044004261736963322028632920323030362DAF
:1000540032303039204A6F65726720576F6C667290
:04006400616D0000CA
:10007000C8EDD1E00895C4E1D1E00895C0E0D1E039
:100080000895CCE3DDE00895E0E0F6EF0895E0E0C8
:10009000F6EF0895FF91EF91EF93FF93EF2FE85460
:1000A000F2E4FA5FE650E8F7EE270895009338018E
:1000B000089500913801089500934A010895009130
:1000C0004A01089500931B0108950C94C1360C94C5
:1000D00049320C94BC320C94D9310C9434320C94C7
:1000E00067340C9446340C944E340C948D350C9437
:1000F000ED3C0C9489320C94EA360C94F136409124
:10010000200108954091220108954091230108950E
:100110004091210108950C9460380C946C380C9433
:100120007C380C9472370C949C3D0C94793D0C9463
:100130007A340C948C360C94CD350C94E6350C94B2
:10014000F73A0C943E3B0C94A3390C9483390C94ED
:1001500094390C9493380C94E6380C94813B0C94AD
:10016000AA3B0C94743B0C949D3B0C94CA360C94A3
:10017000EF3D0C94023E0C94BD3D0C94B93D0C94A3
:10018000C33D0C94C83D0C94BF3D0C940D3E0C94A3
:100190002F3E0C94383E0C944E3E0C94553E0C94DD
:1001A000A73F0C948B400C94FE400C9474410C942B
:1001B0001A410C942E400C94753E0C94833E0C9482
:1001C0000D400E94F6400C94CC3E0E94983E0C9448
:1001D000883F0E94523F0C94B43E0C94FA3EF8942F
:1001E000A0E02A2EA1E03A2EA0E1AEBFAFEFADBF56
:1001F0000E94C8300E94B23D0E9412790E94F938D4
:100200000E944932AFEFA0931001A0933D012092CC
:10021000490120924A0120925C018827789420921B
:100220003901A0913501A4FD0C942F010E9449329F
:100230000E9401040E94EA36D2CFAF91BF91CF91C4
:10024000DF91EF91FF9108950F901F90FF93EF932F
:10025000DF93CF93BF93AF931F920F920895A1E0C6
:100260000E94B631AA270E9442319927A7E10E9435
:10027000B1310E944932A0E10E94B131C4E0DAE01C
:10028000E7E3F7E10E94E635A7E00E94B1310E9462
:100290004E34070420002DD1A6E10E94B131C5E003
:1002A000D8E0E6E0F9E00E94E635D8E1F9E10E9405
:1002B000E635D8E0F9E0CC5FEC5FC833A0F368E73F
:1002C0000E94C1364091200141FD0EC06A95C1F7E0
:1002D00056E142E00E94ED3C0E94C1360E94C136C8
:1002E0005A95B9F70C9491010E9449320E944E34FC
:1002F00000004B6579626F6172642D546573740000
:100300000E94893270917101A0917101A215E1F3EF
:100310002092710190E07A2F0E9434320E94BB3209
:10032000F3CFA0E00E94B631A1E00E944B3899279C
:1003300020923601AA270E944231A5E10E94B131E4
:100340000E944932C0E0D0E0EDE1F4E10E9429369C
:10035000A1E50E94B1310E944E3401018383838361
:100360008383204156522D436869704261736963EB
:1003700032208282828282820000A9EAB4E00AE40A
:100380000D9304EC0D930CE80D9308E20D9302E637
:100390000D9306EA0D93509606EA0D9302E60D932F
:1003A00008E20D930CE80D9304EC0D930AE40D9311
:1003B0007ED2409149014B3008F0442740934901D7
:1003C000642F67FD66276B3008F06AE050E06F939A
:1003D000A3D06F9153955830D1F75ED133D108D166
:1003E0006F9384D16F91423E11F46A95EACF433EF8
:1003F00011F46395E6CF443E21F4643010F064506C
:10040000E0CF453E21F4673010F46C5FDACF6830FE
:10041000F8F04A3E11F0443F19F760934901683003
:1004200039F44A3EE9F673D00E940C1E70D079CFA1
:10043000693039F44A3EA1F66AD00E94D92267D0C9
:1004400070CF65D04A3E61F60E94AC2460D069CF7F
:100450004F934091200142FD29C04F914A3E11F037
:10046000443F41F46093490152D088270E9401041F
:100470004ED057CF413F41F46093490148D088277F
:100480000E94E70344D04DCF423F39F460934901C5
:100490003ED00E94BA1F3BD044CF433F31F460931B
:1004A000490135D00E9421203CCF9ACF4F91413F46
:1004B00031F4609349012BD00E948C0332CF423F2C
:1004C00039F46093490123D00E94502520D029CFD0
:1004D000433F39F4609349011AD00E948B2517D00D
:1004E00020CF443F11F76093490111D00E94D403FB
:1004F00018CF0E944E34FF4156522D436869704216
:1005000061736963322056302E3936000895A09108
:100510002201A030E1F70895A1E0B3E050FDA95F0A
:1005200051FDA25F52FDBA5F452F0E94A679042FAC
:100530004EE20E3409F44CE2651709F442954093FB
:1005400038010E9467340E944E34FF20200040E5AD
:100550000E94BC32452F4F5C0E94BC320E944E3438
:10056000FF202000B3950E946734452F0E94A67992
:100570004E3481F40E944E34FF2020E6E720200014
:10058000B3950E9467340E944E34FF2020E8E92092
:1005900020000FC00E944E34FF2020D0D120200028
:1005A000B3950E9467340E944E34FF2020D2D3209E
:1005B0002000452F0E94187AB3950E94673466E0A8
:1005C00045910E94BC326A95D9F7B3950E94673471
:1005D00066E045910E94BC326A95D9F7B3950E94B6
:1005E00067340E944E34FF202020202020000895F0
:1005F0004AE26A3009F44295409338010E944E3431
:100600000F0F20202020202000000E944E34100FC9
:100610002020D4D5202000000E944E34110F20202D
:10062000D6D7202000000E944E34120F20494E469B
:100630004F2000000E944E34130F20202020202045
:100640000000089548E2693009F44295409338016A
:100650000E944E340F0820202020202000000E94FD
:100660004E3410082020D8D9202000000E944E349B
:1006700011082020DADB202000000E944E341208EE
:10068000434F4E46494700000E944E341308202035
:1006900020202020000008954CE2683009F44295A3
:1006A000409338010E944E340F012020202020204A
:1006B00000000E944E3410012020DCDD20200000CC
:1006C0000E944E3411012020DEDF202000000E9415
:1006D0004E34120144464C41534800000E944E34AF
:1006E0001301202020202020000008953DED2092BD
:1006F00023010E949737409120014470431739F03D
:10070000342F403011F4D3D0F4CFECD0F2CF40915D
:100710002301403071F30895A4E00E94B131C1E09B
:10072000DFE0ECE1F3E10E942936A0E40E94B13160
:100730000E944E341002436F70792050726F6772BE
:10074000616D20746F007091490160E0ACE0671743
:1007500009F4A0E60E94B131B2E1A62FAA0FA60FBC
:10076000AD5F0E94673440E50E94BC32462F47705F
:100770004F5C0E94BC326395683041F70E94EA36B4
:10078000423E21F47030D1F37A95DFCF433E21F41D
:100790007730A1F37395D9CF4A3E19F40E944B7A72
:1007A00008954D3E59F708950E949D3B4F436C6557
:1007B000617220746869732050726F6772616D3F57
:1007C0002000413009F008950E94257A0895A091F3
:1007D0002201A030E1F70E94A4794E3441F00E943A
:1007E000F60420923901A0912301A43F09F099CD8C
:1007F00008D00E94F136A0E00E9442310E944932A6
:10080000E6CF0E9449328827209222010E94167A60
:100810003C9645914E3429F43396F695E795099523
:1008200080CD0E94F90D2092190120925C01209246
:1008300036010E948932A7E20E94B13192E0A09174
:100840004A01A03079F0A33021F4A7E20E94B1312F
:1008500009C0A0E10E94B131A0E4A0930001A0EE84
:10086000A0930101B6E1A0914A01A03079F0B9E668
:10087000A13061F0B2E4A23049F0BFE2A33031F020
:10088000B8E3A53019F0B1E0A63060F0AA270E94C5
:1008900067340E944E34FF20505245535320455335
:1008A00043200000A0912201AD3EE1F70895A0E0B1
:1008B0000E94B1310E944E341500202020202020BB
:1008C0002020202020202020202020202020202028
:1008D00020202020202020200000EEEEF8E00E94C2
:1008E000E6380895ECE0F9E00E94E638089520200B
:1008F00020202020204564697420205361766520E3
:10090000204C6F6164202052756E20202020202012
:10091000202020436F7079202053656E6420205280
:100920006563762020436C656172AA270E94B63108
:10093000A3E00E944B388F93409149010E941D799A
:100940000E9449320E94373199274091220140305C
:10095000E1F70E944E3400002050524F4752414D63
:100960002000409149014F5C0E94BC324AE30E9442
:10097000BC32C3EED1E059D2F1D20E94E579DFD387
:100980008F91A8E8803069F1ACECEEE6F1E18130BE
:1009900031F0ABE48A9545914030E9F7F8CF4DD27C
:1009A00092E0A5E0B1E00E9467340E9446340E94C4
:1009B0004E34FF20494E20500000409146014F5CCC
:1009C0000E94BC324AE30E94BC32BB27AC2DA395E7
:1009D0000E94D9314AE30E94BC32AD2DA3950E94FA
:1009E000D9310895AAE25A2E70E208959927FADFC4
:1009F0009CDFD22CAA27BB27D0923A010E94143741
:100A00000E949737403E11F4AA27F6CF413E11F4D9
:100A1000AFE12BC0423E11F4AA9527C0433E69F4D2
:100A2000A3959B2F0E94F0099A1730F4BE3511F45C
:100A3000AA951BC0AA27B39518C0443E21F4BA95C5
:100A4000B7FDBB2712C0463E21F4B850B7FDBB2707
:100A50000CC0473E11F4B85F08C0453E11F4B39591
:100A600004C04A3E39F5B395AA27A03838F0AFE163
:100A7000BA95B038C0F0AA27BB27BECFA03228F065
:100A8000BE3589F0AA27B395B7CFBF3508F0BEE5CC
:100A90000B2F0D1508F4D02E0D2D015F0B1718F438
:100AA0000B2F0F50D02E9B2F0E94F0099A1708F49D
:100AB000A92FA2CF9B2F4E3E39F4AF93BF930E9434
:100AC000BC09BF91AF918AC14F3E31F4BF930E94E0
:100AD000C709BF91AA2782C1493E11F483D17EC1C3
:100AE0004C3E31F4A03009F489CFAA957BD176C170
:100AF00050912001547009F4C6C0433FD1F4ACECCE
:100B00009CD10E944E340107524543454956452029
:100B100050524F4752414D20592F4E203F006ED129
:100B20002EF46DD20CD35EDF5092D8017ED188278F
:100B300061CF423F39F5ACEC80D10E944E340107C1
:100B400053454E442050524F4752414D20592F4E4D
:100B5000203F000053D156F7ACEC6FD10E944E34C9
:100B6000010753454E44494E472E2E2E202020206B
:100B70002020202000003092360194D120923601AE
:100B800031DFD4CF443FB9F4ACEC57D10E944E349E
:100B90000107434C4541522050524F4752414D208E
:100BA000592F4E203F002AD12EF4BBD2C8D21ADFD3
:100BB0005092D801BBCF413F41F5ACEC3ED10E94F1
:100BC0004E3401075052494E542050524F47524123
:100BD0004D20592F4E203F0011D1B6F4ABE42DD15A
:100BE0000E944E3401075052494E54494E472E2E12
:100BF0002E202020202020202000A2E0A0933601DB
:100C000051D120923601EEDE91CF433671F462E489
:100C10006093F50165E56093F60166E46093F70182
:100C20006DE36093F80158D2E9CE483791F462E45D
:100C30006093F50165E56093F60166E46093F70162
:100C40006DE36093F8010E946C085BD25092D8016A
:100C500018C04637B1F46091F501623499F460E24E
:100C60006093F5016093F6016093F7016093F801DA
:100C70006093F9016093FA0122D261D25092D801B7
:100C8000BDCE8827BBCE423F11F5BF93AF93C9D0ED
:100C9000D9F0ACECD2D00E944E34010753415645F6
:100CA0002050524F4752414D20592F4E203F0000B7
:100CB000A5D046F40E94B1790E94E57940D292DE37
:100CC0007093D801B2D08827AF91BF9195CE433FA2
:100CD000E1F4BF93AF93A5D0B9F0ACECAED00E94D5
:100CE0004E3401074C4F5354204348414E4745531F
:100CF00020592F4E203F000081D026F70E94E57931
:100D00001ED270DE7093D801DDCF413F49F46A2EC8
:100D10007B2EADD0A62DB72D5092D8016FCED2CF5D
:100D20004D3E09F5BF93AF937CD0A9F0ACEC85D0D4
:100D30000E944E3401075155495420572F4F2053DC
:100D400041564520592F4E203F0058D046F7A091DC
:100D50002201A030E1F70E942F31A0E00E94423131
:100D6000AF91BF910895443FE1F45BD029F40E9414
:100D70002F310E9449320895A9E65FD00E944E3477
:100D8000010753415645204348414E4745532042B1
:100D900045464F52452052554E2100000E94EA36EA
:100DA00091CF5091200152FD1CC053FD1AC04C310F
:100DB000C0F04038B0F4AF3171F05A2FAFE10E946B
:100DC00069376A916983AA95A517D9F74883A395CE
:100DD0005092D80113CE0E94693748835092D801AF
:100DE0000DCE0CCE0E9469375A2F5F3121F0498118
:100DF00049935395FACF50E2588308950E94EA36FA
:100E0000493559F0493749F04A3E39F04E3439F006
:100E10004E3629F04D3E19F0F1CF68940895E894CC
:100E20000895A091D801A0320895A8E806D00E94A4
:100E30004E3401054F4B00000895EF93FF9399271F
:100E4000A0934C010E944E34010520202020202038
:100E50002020202020202020202020202020202092
:100E60002020202020202000FF91EF910895A0E075
:100E70000E943C374A3E09F40895423E21F4A030D6
:100E8000B9F3AA95F5CF433E21F4AB3089F3A3958E
:100E9000EFCF403268F3403858F74883AB3009F061
:100EA000A395E6CFC9EDD1E056E149910E94BC324D
:100EB0005A95D9F70E9489324EE511D016F04A951D
:100EC000E1F7542F53954427451719F024D0439543
:100ED000FBCF43E20E94BC320E9489320895CF9337
:100EE000DF935F936F93E894C4E4D2E053E2459FAD
:100EF000C00DD11D50E26991613238F45A95D9F78D
:100F00006F915F91DF91CF91089568946F915F9198
:100F1000DF91CF910895DF93CF934F935F936F93BA
:100F2000C1E4D2E053E2459FC00DD11DDF93CF93C2
:100F3000A39653E26A91613210F45A95D9F7CF9192
:100F4000DF9149910E94BC325A95D9F70E948932AB
:100F50006F915F914F91CF91DF9108950E9424018D
:100F60004F93EAE7FFE0AEE1B2E04591403011F087
:100F70004D93FBCF4F910C941D012045786974204F
:100F800020204E616D65202020536176652020521F
:100F9000656C6F616420202052756E2020000E94D5
:100FA00024014F93EAEAFFE0DECF2020202020201A
:100FB00020205072696E74202053656E64202020BA
:100FC00052656376202020204E65772020000E9405
:100FD00024014F93EAEDFFE0C6CF2041626F7274A7
:100FE0002020202020202020202020202020202001
:100FF0002020202020202020202020202000E7DF8B
:10100000ACEC1BDF0E944E34010552454345495666
:10101000494E472E2E2E000020923A0182D08FD0CA
:101020009927ECECE0934C01E3EEF1E0EE2EFF2E7D
:1010300041E10E9460385CE00E947C384B31B9F19C
:101040004A33D1F70E947C384B3189F1403218F095
:1010500041935A95B9F7403228F00E947C384B31C1
:1010600031F1F9CFEEE1F2E0EE2EFF2E53E2EE2D5C
:10107000FF2DB396EE2EFF2E0E947C384B31B9F037
:101080004032D0F3433299F006C00E947C384B3195
:1010900071F0403248F041935A95B9F70E947C387C
:1010A0004B3129F04032D0F793959036F9F60895F8
:1010B000A3E2BA9FA1E4B2E0A00DB11D0895BF93D1
:1010C000AF93F6DFC8E8D1E053E249914D935A95CA
:1010D000E1F7AF91BF910895BF93AF93E9DFC8E8FF
:1010E000D1E053E24D9149935A95E1F7409188013F
:1010F0004093F901409189014093FA01AF91BF916A
:101100000895BF93AF934F935F93D2DF139640E25E
:1011100050E24D935A95E9F75F914F91AF91BF918E
:1011200008950E9424014F9340E2A1E4B2E0CDEF84
:10113000DCE04D932197E9F74F910C941D010E943B
:1011400024014F9341E0A1E4B2E0C0E3D42FDA5090
:1011500010F0C395FCCFD65CCD93DD93C0E2CD9368
:1011600090964395403689F74F910C941D01425259
:1011700045414B004F564552464C4F570044495647
:10118000494445202F30005351522046524F4D20A4
:101190003C3000434F4E5354414E5420544F4F2047
:1011A0004249470057524F4E4720455850524553E9
:1011B00053494F4E0053594E544158204552524FB7
:1011C0005200554E4B4E4F574E204B4559574F529C
:1011D000440057524F4E4720464F524D4154004213
:1011E0004144204C494E454E554D424552004E45D6
:1011F000585420572F4F20464F52005245545552B5
:101200004E20572F4F20474F53554200544F4F20E9
:101210004D414E5920474F53554200544F4F204D9A
:10122000414E5920464F5200493243204552524FB9
:101230005200554E4B4E4F574E204552524F520082
:1012400044464C415348204552524F52004F55544A
:10125000204F4620415252415900494E434F4D5074
:101260004C45544520504152004B4559574F52442C
:10127000204953204D495353494E470057524F4E32
:10128000472042434F505920004F5554204F46208D
:1012900053435245454E0043414E4E4F5420435216
:1012A000454154452046494C45004D454D4F525906
:1012B0002046554C4C0046494C45204E4F54204644
:1012C0004F554E440050414745204E4F5420494E03
:1012D0002046494C45005041474553204E4F54202D
:1012E000494E2052414E4745004E4F5420494E2012
:1012F0004752415048494353204D4F4445004E4FBB
:101300005420494E2054455854204D4F4445004EDA
:101310004F205553522046494C4500535243204FCD
:101320005554204F462053435245454E00444553A3
:1013300054204F5554204F462053435245454E00AC
:1013400057524F4E47205350524954450057524F21
:101350004E4720454550524F4D20414452004E4F7C
:10136000205052472046494C4500584D4F44454D6A
:10137000204552524F520000BE3508F00895BF93E9
:1013800023D0B395BE35E1F7BCDEBF91D8CEBE35D4
:1013900008F00895BF93AF93AB2FAA95BDE508D091
:1013A000BA95BA17E1F7B395ACDEAF91BF91C7CE4E
:1013B0000E9424017DDE1396ED01B0E2A991AAA35B
:1013C000BA95E1F70C941D010E94240171DE139679
:1013D000ED01B0E2ABA1A993BA95E1F70C941D0120
:1013E0000E94240165DEED0193964E914132E8F3AF
:1013F0004038D8F7AC1BBC0B9A2F925097FD992719
:101400000C941D01DCC0CAEFDCE02A922A9280E035
:101410002F92AA27BB27442771917032E9F37038C5
:1014200088F77A3379F37C3111F07E3121F4A19180
:10143000BB27719122C07D3111F07F3121F4B19130
:10144000A19171911AC07C3160F4572F2E01EF01E8
:101450005F93452FAA27BB27FE01E201DDCF87E07E
:10146000BEC0703398F07A3388F4403810F086E0CC
:10147000B6C0A72FA053BB2771914F3709F41AD1DB
:10148000AA93BA9340E8CBCF85E0A9C07134A0F00D
:101490007B3590F4403810F086E0A1C07154770F8E
:1014A000EF93FF93E0EAFCE0E70FF21DA191B19109
:1014B000FF91EF917191E1CF7D3251F44F3711F4EB
:1014C0004427AACF20F4403210F04FE7A5CF4DC0FB
:1014D000783231F471E07F93AA27BB27472F9CCF46
:1014E000793209F03CC05F915C3160F5B991A99106
:1014F0000FE71AE0050F121D0F931F93089527C0E1
:1015000028C019C01AC09DC11AC0AEC146C27AC255
:101510008FC2A9C2B2C2B3C2B5C294C203C3E6C1EC
:1015200018C11AC1ECC101C2AAC1BFC1C4C147C21E
:1015300058C208C34BC3BCD00CC0CBD00AC0B095B6
:10154000A09507C063D0803009F049C0CCCF86E0B9
:101550000895AA93BA93AA27BB2742E05DCF4F37DD
:1015600020F44F3010F086E03AC0608132E27C33E4
:1015700039F46E33C1F133E26D33A9F131E234C095
:101580007E3329F435E26D3371F134E22DC036E259
:101590007D3351F137E37B3239F138E37D3221F18C
:1015A00039E3733209F13AE47A32F1F03BE47F3205
:1015B000D9F03CE47532C1F03DE47632A9F05F9198
:1015C000503021F05F3130F021D0F9CFB991A9919D
:1015D0003197089586E05F915030C1F3FCCF4F9171
:1015E0004030E9F708953196732F5F91A72FB52FFB
:1015F000A07FB07FBA1720F009D0803081F7F5CFF7
:101600005F937F93AA27BB27472F06CF5F934F9304
:1016100019910991B991A99127E1352F3F70330FA5
:10162000330F230F3BE0321D2F933F9308953BC0B0
:10163000000000000000F2D036C000000000E7D03B
:10164000A150A17030C0F2D0A150A1702CC0EED03A
:101650002AC000000000E2D0A150A17024C0D7D061
:1016600022C0000000003ED01EC00000000039D0A3
:101670001AC000000000A02BB12B15C000003DD007
:1016800012C000000000A2D00EC0000000009ED0DA
:10169000A22FB32F08C0A023B12305C0000003C0B0
:1016A000000000000000AA93BA934F915F91089543
:1016B000B7FF0895A095B095A30DB21D0895AA9304
:1016C000BA93089517FF089500951095030D121D04
:1016D0000895AB2B29F0B7FBA1E0BB270EF41297BE
:1016E00038CFF2DF2B2F2127A00FB11F27FD089540
:1016F0002B2F212727FD82E008950CD0A22FB32F96
:10170000BF770EF4D7DF37FD03C0452B09F40895EA
:1017100082E0089577D0CCDFB19F402D512DA09F5E
:10172000202D312DA19F300D411D521DB09F300D38
:10173000411D521D089508E611E0B03818F0A00FC1
:10174000B11FFBCFA017B10718F0A01BB10BFACF48
:1017500008950AE5A01BB20901D0FBCEECDFFF9390
:10176000EF93E8E6F3E80AE510E0A017B10748F4C4
:10177000E00FF11FEA1BFB0BA491EF91FF91BB2738
:10178000089504EB10E0A017B10778F40AE510E023
:10179000E01BF10BEA0FFB1FA491EF91FF91BB2718
:1017A000A095B095A30DB21D08950EE011E0A0170D
:1017B000B10728F4E00FF11FEA1BFB0BEDCF0EE0A1
:1017C00011E0E01BF10BEA0FFB1FD6CF212F202BDE
:1017D00011F483E0089516D022273327442751E1DE
:1017E000441FAA1FBB1F5A9551F0221F331F4FEFF2
:1017F000201B310BA8F7200F311F40E0F1CF0EF472
:1018000059CF08952B2F212727FB52DF5BCF0A27C3
:101810001B27AA27BB27012B89F00895B058105821
:10182000A01BB10BAA27BB2748F00895B058105849
:101830000A1B1B0BAA27BB2708F00895A1E0B0E004
:10184000089584E0B7FD089588270A2F1B2FB2E082
:10185000AA27232D3327021B130B20F0A3952B0F50
:10186000321DF9CFBB2775CE4F935F938D010E9438
:10187000083952DFA42FB52F5F914F916ACE8D01A9
:10188000023039F420925C01A2E0A0933F01BB2713
:1018900060CE013031F4A0913F01A03011F43092BC
:1018A0003F01A0913F01BB2754CEAEBD0E940E1A4E
:1018B000AEB5BB274ECE10914A01103011F08CE12D
:1018C000089504EC12E0A017B10710F082E108952A
:1018D000FF93EF93FDE0ECE3EA0FFB1F68940E9497
:1018E0009338EF91FF91A42FBB2733CEB0937301B0
:1018F000A0937201DF93CF930E941A1A28C0BF3FB2
:1019000071F0A09378010E94B922803021F0AFEFEE
:10191000BFEF88271ECEA42FBB270C94A90A0E94D4
:10192000BE228827B42FAA2714CEDF93CF93FF932C
:10193000EF93BF3FC1F4A0FD0DC00E94B6228030DE
:1019400019F08827CC27DD27DE01EF91FF91CF9199
:10195000DF91FFCD0E94B622803019F08827EE2754
:10196000FF27DF01F2CFA09378010E94B9228030D7
:1019700021F08827AA27BB27E8CF7F9377270E94EB
:10198000C122DF3F31F4CF3F21F4A72FBB277F9146
:10199000DCCF7395703899F7F8CFA770A06CA0933F
:1019A0007C00A0917A00A064A0937A00A0917A00B4
:1019B000A6FDFCCFA0917800B0917900CACDBB30D4
:1019C00020F4BA3028F0A83C18F0AFEFBFEFC1CD3B
:1019D000DF93CF93C8EDD1E0CA0FDB1FA881BB27EF
:1019E000B6CFB33018F4B23010F0A7FDF8CDDF93C6
:1019F000CF93CCE3DDE0CA0FDB1F0E94793DA62F19
:101A0000BB27A5CFB03061F4AF3F79F0A770A395A5
:101A1000B0B1B695AA95E9F7AA27AA1FBB2799CD19
:101A2000BA2FA0B1AB23BB2794CDA0B1BB2791CDDA
:101A30007091650177700E94EF3D8030D1F4BB2733
:101A4000A52F87CDCF93DF93CA2FDB2F0E942F3E88
:101A5000DF91CF91803019F4BB27A42F7ACDAA272C
:101A6000BB2782E2B8CD7A2F0E940D3E803009F468
:101A700070CDAA27BB278FE0AECDBB276ACDAB2F99
:101A8000BB2767CD0F930A2FAA27BB27003019F475
:101A9000A091220145C0013029F4A0912201A0307B
:101AA000E1F33EC0023039F4A0912201A030E1F709
:101AB000A091230135C0033019F4A091200130C05A
:101AC000043039F40091200100FD119602FD1197B8
:101AD00027C0053039F40091200101FD119603FD66
:101AE00011971EC0063049F400912201023E09F40C
:101AF0001197033EA9F4119613C0073049F40091E1
:101B00002201043E09F41196053E51F4119708C0D4
:101B10001F93109122010117E1F71F91A02FBB27FE
:101B20000F9117CDBB27A13021F4A0916D01A39592
:101B300010CDA23021F4A0916E01A3950ACDA09101
:101B40006F0107CDCF93DF93EF93FF936F927F9257
:101B50004F930E94833E4030A9F0342F3395ED011E
:101B60000E94121A803071F521963E011A2F00272B
:101B7000A02F0E94F8400E94CC3E141721F003953C
:101B80000317B1F71CC0E3010E94121A8030D1F490
:101B9000A03091F02A2FA02F0E949C41E3012196B2
:101BA000E8E8F1E00E94121A803061F4B191AB17BD
:101BB00031F721962A95B1F7A02FBB2702C0AFEFCE
:101BC000BFEF88274F917F906F90BFCECF93DF9369
:101BD000EF93BA2FAA27C0E0D8E0CB27BB0FEC2F9A
:101BE000EE0FAA1FDA95C9F7EF91DF91CF91BB27CE
:101BF000B0CCFCE0E0EAA0E0B4EBA193BA95E9F741
:101C0000F1E0E8E6B0E1A193BA95E9F7FDE0ECE395
:101C1000B0E0A193A193A193BA95D9F7DD24CC2488
:101C200020921B0120921901AEE0A0933801ACE391
:101C3000A0935001AEE2A0935101AFEFA0937701C2
:101C4000A0931001209213010E94493220925C015E
:101C5000A2E0A0933F01A6ECA0937A004091490135
:101C600040934601409343010E941D799C2D0E94A0
:101C70002D7921D0803039F4AC2DAF35B8F39CE00C
:101C800020925C010895C0926D01D0926E01809304
:101C90006F01813051F020925C01409177014F3506
:101CA00020F4DD24C42E8827E1CF9CE020925C0143
:101CB0000895F7012AC0F1E0E0EB20923601882771
:101CC000AD2DBB27AB1709F171917F3FD1F07C316E
:101CD000D1F07E31C1F07D31A9F07F3199F07732BA
:101CE00081F0723241F471917F3F59F0773249F0BF
:101CF0007232C9F7E9CF7A3339F7B395AB1721F7C9
:101D000004C02FC071917191DFCF7091390170FFC4
:101D100005C081E07E7F70933901089572FF11C084
:101D2000AB7F70933901A0914A01A53011F0A0302A
:101D300011F40E94101DA0FF04C00F900F9081E0CD
:101D400008950E94973770911301703039F0A09177
:101D50001001DA94209213010C94771271917F3F55
:101D600019F4DD24C394089577FD2BC0703269F215
:101D70007A3311F4D394C9CF773219F27134D8F091
:101D80007B3528F070527134B0F07B35A0F4672EAB
:101D90000E9495177D3379F436DB803069F4762D17
:101DA0007154770FDCE0C0EAC70FD21DA993B99335
:101DB00081CFEF91FF9187E00895703810F487E0AC
:101DC00078CF7F01E9EEF72FFF73EF0FFEE0F21DF2
:101DD00009944DC0F7C0DDC270C142C115C35DC3D7
:101DE0007FC768C36DC375C33AC0C8C6E6C675C3AE
:101DF000DFC3FAC234C464C4B5C1A6C4B6C4BBC48C
:101E000026C2D2C2C0C4CBC4D2C48FC587C10BC145
:101E1000B4C268C113C5D5C428C014C535C58BC2AA
:101E200005C3FCC5ECC751C65DC662C6B0C1E4C6F9
:101E300035C7BDC763C672C697C249C594C65CC1E3
:101E4000BEC2D4C332C3CEC4D0C47AC1B2C176C676
:101E5000CFC188E0089584E1089583E10895703C3E
:101E600010F00C948B190C9450180C946A180E9462
:101E700099179CE0732C20923601B191B032E9F3AE
:101E8000BA3321F0B73211F0BF3F59F4319770FCEB
:101E90000E94893240913601443010F00E94B93DD1
:101EA00009CFBB3311F47724E8CFBC3291F44091D1
:101EB0003601403031F40E94BB32BA2DB770D9F7E9
:101EC00006C00E94BB32B0913701B770D1F77724BA
:101ED000D4CF732CB332C9F42092780120927901C7
:101EE00092DA4A2F40933601443018F4433001F41B
:101EF000C4CF0E94BD3D683051F5509136015E7FE0
:101F00000E94BF3D683119F5B8CFB03411F5DCD768
:101F100040913601433018F40E946734AECF39F453
:101F2000A0937801B0937901A0933701A6CF5FEF1A
:101F30000E94BF3D683259F45A2F0E94BF3D68325B
:101F400031F45B2F0E94BF3D683209F496CF8FE0D9
:101F50000895B13229F457DA9A2F8FCF97CF8DCFCA
:101F6000B23241F441914F3FC9F34232C1F30E9472
:101F7000BC32F8CFB63291F446DAB33010F082E1D9
:101F80000895CCE3DDE0CA0FDB1F4991403029F012
:101F90000E94BC321196B330C0F36FCFB53229F432
:101FA00032DA4A2F0E94BC3268CF31972CDA803067
:101FB00009F00895903818F40E94D9315ECF0E943C
:101FC00034325BCF703CB8F4A1E030D7B0914A0115
:101FD000B63019F00E9449326CCEA13029F00E942F
:101FE00083390E94943965CEB0917801B130C9F33C
:101FF0000E9483395ECEA2E019D7A23081F5A0E815
:10200000B2E060917801C0917A01D0917C01CA1749
:10201000DB0738F4ACE3BDE0CA0FDB1F0E949C3D38
:1020200048CE82E10895A2E001D7A030C1F0A130EE
:1020300059F0A0917A01A770AA0FB0913801B7703A
:10204000A295BA2BB0933801A0917801A770AA0F7E
:10205000B0913801B07FBA2BB09338012ACEFDCEB3
:10206000703C10F00C945119A3E0E0D6A33018F1A5
:10207000A0917801B0917901A0937201B09373019E
:10208000A0917A01B0917B01A0937801B09379017E
:10209000A0917C01B0917D01B03011F4A03051F0DD
:1020A0000D010E941A1A0E94F217D001803021F40B
:1020B0001197F2CFFECDD1CE0895733C09F4F9CD3E
:1020C000A5E0B4D6A43068F0C4D77F93ECD6E093F3
:1020D0006B01F0936C010E94CD357F9170933801B4
:1020E000E8CDBBCEA1E0A2D6A130D8F340917801D3
:1020F000417040931901DDCDA5E098D6A43068F079
:10210000A8D77F93D0D6E0936B01F0936C010E9427
:10211000E6357F9170933801CCCD9FCEA5E086D671
:10212000A43068F096D77F93BED6C0936B01D0934E
:102130006C010E94F73A7F9170933801BACD8DCE31
:10214000A5E074D6A43068F084D77F93ACD6C09352
:102150006B01D0936C010E943E3B7F9170933801DC
:10216000A8CD7BCEA3E062D6A23080F072D77F9359
:10217000B0917801A0917A01A0936B01B0936C01AA
:102180000E947A347F917093380193CD66CEA5E09A
:102190004DD6A43068F05DD77F9385D6E0936B0170
:1021A000F0936C010E948C367F917093380181CD41
:1021B00054CEA0914A01A03011F08CE10895A1E025
:1021C00035D6A130A8F3A0917801B0917901CCE384
:1021D000DDE0CA0FDB1F409138014F93AF92BF92F1
:1021E0000E94813BBF90AF904F914093380161CDE9
:1021F000A0914A01A03011F08CE108957FD6C093E0
:102200007201D093730191D67C32F9F4A1E00FD61C
:10221000A13070F2A0917801B0917901CCE3DDE0BA
:10222000CA0FDB1F409138014F93AF92BF920E94BB
:10223000AA3BBF90AF90C0917201D09173014993B6
:1022400029924F914093380134CD87E032CDA0914F
:102250004A01A03011F08CE1089550D6C09372016C
:10226000D093730162D67C3281F7A1E0E0D5A13032
:1022700009F0F3CDFF93EF93AF92BF9240913801F5
:102280004F937F934F70409338010E94D41BC1E05D
:10229000D2E0ECE1F5E10E942936C0913801C29507
:1022A000C09338010E944E3403020000A0917801CF
:1022B000B0917901CCE3DDE0CA0FDB1FA6E14991C3
:1022C000403230F0403820F40E94BC32AA95B9F771
:1022D000772761E025D00E94F61B623079F4C09127
:1022E0007201D0917301799329927F914F9140931C
:1022F0003801BF90AF90EF91FF91DBCC7F914F9170
:1023000040933801BF90AF90EF91FF91C09172015F
:10231000D09173014FEF49934993CBCC87E0C9CC5F
:102320000E9442188827603009F408950E946220B4
:10233000882762E00895A3E079D5A230A0F089D67D
:102340007F93D0916C01C0916B01F0917801E09185
:102350007A01E0936B01F0936C010E948C367F91BF
:1023600070933801A6CC79CDA4E060D5A43021F4D7
:102370009AD50E948D359DCC70CDA1E057D5A13066
:1023800090F0A0917801A295AA0FAF7EA0931B01B7
:1023900090CCA1E04BD5A13030F0A0917801A150B4
:1023A000CA2EDD24089559CDA1E040D5A13030F0EA
:1023B000A0917801A150A09377017BCC4ECDA7E0EE
:1023C00035D5A230D8F3C8E7D1E0E881EF70F1E06D
:1023D000BA81B770BB0FB295B193EF702296AA95F0
:1023E000A130B1F766CC39CDA1E020D5A130D8F32A
:1023F000A0917801A7700E944231A0914A01A730B4
:1024000010F40E94493255CCA1E010D5A13068F0FB
:10241000A0917801B0917901B03019F4A03009F49D
:1024200048CC0E94C1361197F7CF17CD20925C019E
:10243000A2E0A0933F01A3E0F9D4A33058F1CCE38C
:10244000DDE0A0917801B0917901B33020F5AC0FB7
:10245000BD1FA0935E01A0936001B0935F01B09394
:102460006101AC1BBD0B00907A010A94A00DB21D56
:10247000A00DB21DB33078F4AC0FBD1FA093620164
:10248000B0936301A0917C01A0935C013092640140
:1024900020923F010ECC82E10CCC703C28F42092BB
:1024A0005C01BF91BF910895C1C645D5AB2B09F41E
:1024B00028CC00CC703C10F00C946B193AD5FACBB8
:1024C000703C10F00C94AB19F701FED40E946734F5
:1024D000F1CB31D50E94CA36EDCBA2E0A7D4A13012
:1024E00019F0A23021F1B9CCA0917801AA95AF35AD
:1024F00010F08AE0DECBB0917001BB3010F08DE0BF
:10250000D8CBAF93CCEFDCE0A5E0AB9FC00DD11DE5
:10251000B395B0937001BD2DB395B068B993BC2D40
:10252000B993B0914901B993DD24CF9008954091BA
:1025300078014A950E94A6794E3469F4A0917A01F7
:10254000B0917B01B630A8F6F695E795EA0FFB1F30
:1025500038960995AECBA0917A01AA95AF3548F689
:10256000B0917801BA95B770B0934301B091700102
:10257000BB3010F08DE09DCBAF93CCEFDCE0A5E05D
:10258000AB9FC00DD11DB395B0937001BD2DB39518
:10259000B068B993BC2DB993B0914601B993DD24CD
:1025A000CF9040914301409346010E941D790895C8
:1025B000C0D4B0917001B03011F48CE00895BA9598
:1025C000CCEFDCE0A5E0AB9FC00DD11DB093700156
:1025D000B991B7FFF2CFBF77DB2EC99049914093F5
:1025E00046010E941D79089587E00895A2D49DD4E4
:1025F0007134D0F37B35C0F77154770F672E95D4C3
:102600007D3391F70E94030A803009F00895DCE0E1
:10261000C0EAC60DD21DA993B99387D4733C21F7A4
:102620000E94030A4A2E5B2E803009F00895B09173
:102630007001BB3010F08EE00895CCEFDCE0A5E037
:10264000AB9FC00DD11DB395B0937001BD2DB39557
:10265000B993BC2DB9936992499259922BCB69D405
:10266000B0917001B03011F48BE00895BA95CCEFC1
:10267000DCE0A5E0AB9FC00DD11DB991B7FDF4CF53
:10268000BF77B0936A0159907991BCE0A0EAA70F97
:10269000B21D0D911D91030D121D1E930E93A99154
:1026A000B99111960A1741F41B1731F4B0917001DA
:1026B000BA95B0937001FECAC52CD0906A010895F6
:1026C000A0914A01A03011F08CE1089532D4BFEFFF
:1026D000B0938801B191B032E9F34B2FBF3F21F4A1
:1026E0000E9489323197E6CABA33D1F3BB3391F3F2
:1026F000BC3231F40E94BB32BA2DB770D9F7EACFA1
:10270000B23241F441914F3F59F3423219F30E94E2
:10271000BC32F8CFB134B0F0BB35A0F4B154BB0F2C
:10272000B0936A01B081B13418F0BB3508F40AC027
:1027300005D4DCE0C0EA10916A01C10FD21DA99353
:10274000B993C8CF87E00895F6D3803009F0B2CAB4
:102750004A2F4B2BE1F340912E014030E1F34091A1
:102760002E014030E1F71197F3CFE5D3A0932F016D
:10277000B0933001EDCFC2D3A0912F01A993A091C6
:102780003001A99397CAD7D34A2F0E946038CED37D
:102790007C3221F4CAD30E94030AF6CF8BCA0E946E
:1027A0006C38A42FBB27AAD3A993B99383CAF70186
:1027B00098D34A2FD73020F4C03D10F40E94383E01
:1027C00079CAF7018ED35A2FAC2FBD2F70916501B6
:1027D00077700E94023E0E94C1360E94C1360E945C
:1027E000C13668CAA8D3A1B965CAF7017AD3D03077
:1027F000B1F4BC2FB770B39577276FE7A0FD70E8F1
:10280000A0FD6FEF77FB770F70F967FB660F60F93C
:10281000BA95C1F702B1072B062302B94BCAD130D2
:1028200041F4B2B1C095BC23C095CA23BC2BB2B948
:1028300041CAD230E9F70E94FC193CCA7CD30E94FD
:102840004B3838CA5BD3C0937201D093730109919E
:10285000199110586AD37C32A9F443D3B058D05898
:10286000C017D10710F00C2F1D2FA017B10710F4BF
:102870000A2F1B2FD0917301C09172011058099338
:10288000199318CA86E00895A0914A01A63029F04C
:10289000A370A03011F08CE1089530D3C093720181
:1028A000D093730142D37C3269F70ED3C8EDD1E0E7
:1028B0007EE17B9FC00DD11DCA0FD21DBB27A88111
:1028C000D0917301C0917201A993B993F3C9A091FA
:1028D0004A01A370A03011F08CE108950FD3C0938A
:1028E0007201D093730121D37C3261F6EDD2C8ED31
:1028F000D1E07EE17B9FC00DD11DCA0FD21DA2EB9E
:10290000CA0FA2E0DA0FBB27A881A695BA2FA77736
:10291000B295B078AB2BBB27D0917301C0917201F7
:10292000A993B993C7C986E00895E8D2C09372010C
:10293000D0937301FAD27C32B1F7C6D2C8EDD1E0A0
:1029400070914A017770703021F5AF93BF93A695CF
:10295000B6957EE17B9FC00DD11DCA0FD21D788137
:10296000BF91AF91A0FD7695B0FD7695B0FD7695BF
:10297000A2EBB2E0CA0FDB1FA88170FFA295A6955B
:10298000A770BB27D0917301C0917201A993B9932D
:1029900091C97130B9F4AF93A695A695A69575E146
:1029A0007B9FC00DD11DCA0FD21D7881AF91A2FDB2
:1029B0007295A1FD7695A1FD7695A0FD7695717035
:1029C000A72FDECF7230A1F4AF93A695A6957EE136
:1029D0007B9FC00DD11DCA0FD21D7881AF91A1FD83
:1029E0007295A0FD7695A0FD76957370A72FC8CF40
:1029F000733071F4AF93A6957AE27B9FC00DD11D21
:102A0000CA0FD21D7881AF91A0FF7295A72FB8CFC2
:102A1000AF93A695A695A69570E1C2CFA0914A0165
:102A2000A63029F0A370A03011F08CE10895A3E046
:102A3000FDD1A33080F0A0917801B0917901B3303D
:102A400010F082E10895B23039F4A73F28F082E116
:102A5000089581E2089501CACCE3DDE0CA0FDB1FCF
:102A6000C0935201D0935501AC81A03091F3AE31A7
:102A700080F7BB81B03069F3B73158F7C091780166
:102A8000D09179012596BA9F000C111C000C111CE5
:102A9000C00DC11DD330E8F6D0917A01C0917C0100
:102AA000C0935401D0935701CF3F51F0DF3F41F025
:102AB000CA0FCA95CE3138F4DB0FDA95D73118F446
:102AC0000E941C3CF6C886E10895A0914A01A030FE
:102AD00011F08CE108952DD2A0913901A460A0934A
:102AE0003901E8C8A0913501A062A0933501E2C880
:102AF000A0913501AF7DA0933501DCC8A3E096D14C
:102B0000A33009F0AAC90E94B922403310F08EE127
:102B100008950E94CD228030D9F7CBC8A3E086D19A
:102B2000A33009F09AC90E94B922403310F08EE117
:102B300008950E94D0228030D9F7BBC8A3E076D197
:102B4000A23019F0A33021F088C9A4E1A0937C0140
:102B50000E94C722803009F4ACC808950E94CA229E
:102B6000803059F4A6C8A1E061D1A13009F075C93F
:102B70000E94B922443191F38EE10895A2E056D12A
:102B8000A23009F06AC9A0917801B0917901409111
:102B90007A01CCE3DDE0403041F0D395413029F0BB
:102BA000D395423011F082E108950E94983E0E9430
:102BB000883F803009F008957CC8A2E037D1A23068
:102BC00009F04BC9A0917801B091790140917A0147
:102BD000CCE3DDE0403041F0D395413029F0D3958E
:102BE000423011F082E108950E94523F0E94B43EAB
:102BF000803011F308954EC0F7014AD1A0937401BB
:102C00000E94BD3D6830B9F790FF28C0592F0E943F
:102C1000BF3D603481F7A030C9F0DDE0CCE34091E6
:102C200074014B0F4A1BC40FD21DA13039F00E9412
:102C3000C33D603579F55883AA95EFCF0E94C83D12
:102C4000683541F558830E94B93D34C80E94C33DA0
:102C50005030A1F350937401A52FDFCF592F0E945C
:102C6000BF3D6831B9F43A2FDDE0CCE34091740107
:102C70004B0F4A1BC40FD21D5881503011F4303015
:102C800031F00E94BF3D683229F4AA9569F70E948D
:102C9000B93D10C88FE00E94B93D08954CD1A09372
:102CA0007801B093790142D17C3249F431963DD11B
:102CB000723239F031970E94030A94D1F4CF0C9408
:102CC0005A0E7191723231F07F3F21F0BB27A72F4E
:102CD00089D1F7CF7081E7CFA430A9F40C949E1866
:102CE000A7E0A4D0B0917801B0935801B13069F059
:102CF000B23041F1B43081F3B53071F3B63061F3E5
:102D0000B33009F43DC085E10895A730E1F7C8E785
:102D1000D1E0BA81B0935501BC81B0935201BE811C
:102D2000B0935601B885B0935301BA85B09357015B
:102D3000BC85B09354010E94A339803009F00895F6
:102D40000C94590EA630F9F6C8E7D1E0BA81B093D9
:102D50005501BC81B0935201BE81B0935601B88534
:102D6000B0935301BA85B0935401BB85B09357011A
:102D70000E94A339803009F008950C94590EC3CFF6
:102D8000A430E9F7C8E7D1E0BA81B0935201BB8122
:102D9000B0935501BC81B0935701BE81B0935401EB
:102DA0000E94A339803009F008950C94590EA09127
:102DB0004A01A03011F08CE10895F70192D0C09340
:102DC0007801D093790150917401A51708F45A2F16
:102DD000A8E8B1E0503071F04D91A0937501B09327
:102DE0007601A42FBB27FED0A0917501B09176018A
:102DF0005A95F0CFAA27BB27F5D00C945A0EA09174
:102E00004A01A03031F0A43021F0A63011F08CE15D
:102E10000895A1E00BD0A13040F0A09178014A2F95
:102E200043700E94ED3C0C94590E17C8F701A03076
:102E300009F40895DF93CF93C8E7D1E040E05A2F1B
:102E4000503029F4A42F7F01CF91DF910895DF93B3
:102E5000CF934F935F930E94030A5F914F91CF915D
:102E6000DF91893121F488277F01A42F0895A99348
:102E7000B99343955A95503019F371917032E9F333
:102E80007C3229F33197A42F7F01CF91DF910895F0
:102E9000A3E0CCDFA33009F590917801B0917A01DD
:102EA000A0917C010895D0917801C0917A01F091B0
:102EB0007C01E0917E01C0935201D0935501E093D3
:102EC0005301F09356010895A2E0B1DFA23029F436
:102ED000B0917801A0917A010895AF91AF910C94CF
:102EE0002D0FA2E0A4DFA230C1F7C0917801D091EC
:102EF0007901A0917A01B0917B010895F70115D075
:102F0000713478F07B3538F47154770FDCE0C0EA27
:102F1000C70FD21D0895713620F07B3710F471561B
:102F2000F4CF8F918F9187E0089571917032E9F31A
:102F30000895F7010895F7010C94030AEF93FF93A6
:102F40000E945637EC2FFD2F00E00E94F63670915C
:102F50003901713011F4872F09C04A3EE9F400931A
:102F60007401003031F4AA27BB278827FF91EF9125
:102F70000895C8E8D1E0A191A9930A95E1F7AFEFD0
:102F8000A9930E94471AE0EBF1E00E94030A8D0129
:102F90000E942D79D801E9CF4C3E49F40030A9F2C6
:102FA000AA940E945637A0E2A8830A95CECF403259
:102FB00028F24B3718F6AA2DAD3100F60E94BC322C
:102FC0000395C3CF92E0BB27AC2DA3950E94D931C6
:102FD0004AE30E94BC32BB27AD2D0E94D9310E942A
:102FE000BB320895DF93CF93BF93AF93A091780145
:102FF000B0917901B33098F4CCE3DDE0CA0FDB1F68
:10300000AF91BF91A883C0917801D09179012196A9
:10301000C0937801D0937901CF91DF910895B45096
:1030200090F0AA0FBB1FB33070F4CCE3DDE0CA0F01
:10303000DB1FAF91BF91A993B993C0917801D09153
:1030400079012196E5CF82E1AF91BF91CF91DF91D8
:10305000089570913801A0FF0895A33059F450915C
:103060007C015F70550F707F572B70913801509322
:1030700038010895A53019F450918001F2CF509194
:103080008401EFCF0E94D322403011F466270895C7
:10309000409380010E94C422413009F066270895C0
:1030A000A2E0C4DEA130A0F0B1E0A13011F0B091F7
:1030B0007A01A0917801A150A0931001B093110161
:1030C0000E94C136B0931201209213010C94590E44
:1030D0000C942D0FA3E0AADEC0917801D091790164
:1030E00040917A0108EC1AE028ED31E0A23080F33B
:1030F00019F41CD00C94590E60917C01F0917B0165
:10310000F170E0917A014CE3E40F4DE0F41F4427A5
:10311000C40FD21D41910AD041914038C8F34058A4
:10312000C40FD21D6A9551F70C94590EC017D107E0
:1031300020F4DE01A20FB31F4C930895FF93EF9389
:103140000CE310E120EA3CE0B0917801B43019F5CD
:10315000E8EDF1E0A0917A01B0917B01BF70AE0F74
:10316000BF1FC0917C01D0917D01DF70CE0FDF1FAA
:10317000E0917E01F0917F01A217B30740F4C217DE
:10318000D30728F4319718F00D900992F5CFEF91FD
:10319000FF910C94590EB53009F5E8EDF1E0A091DE
:1031A0007A01B0917B01BF70AE0FBF1FECE3FDE071
:1031B000C0917C01D0917D01DF70CE0FDF1FE091C7
:1031C0007E01F0917F01A217B30708F7C017D1075E
:1031D000F0F63197E0F20D900992F5CFB63011F587
:1031E000ECE3FDE0A0917A01B0917B01BF70AE0FDE
:1031F000BF1FE8EDF1E0C0917C01D0917D01DF704F
:10320000CE0FDF1FE0917E01F0917F01A017B10783
:1032100040F4C217D30728F4319718F00D900992A3
:10322000F5CFB5CFEF91FF9185E10895A3E0FEDDE5
:1032300040914A01463021F04430E1F00C94590E9F
:10324000A33071F5AAE8B4E04EE150917A015F73C2
:10325000459FA00DB11D009038014091780150911B
:103260007C015093380155270E9453390092380150
:103270000C94590EA230A1F4E0917801F6EFA0E889
:10328000B7E050917A015F77A50F5AE060E844916A
:103290004C93F395A60FB21D5A95C9F70C94590E8D
:1032A00017CFA2E0C3DDA23011F00C942D0F0E94C5
:1032B000B922803009F00895403121F0483111F0F1
:1032C00083E208957091780190917A019A950E9415
:1032D000D4210C94590EA2E0A9DDA23011F00C9477
:1032E0002D0F0E94B922803009F008954C3F11F053
:1032F00087E10895709049017091780190917A0169
:103300009A95909349010E949E21709249018030C4
:1033100001F00C94590EA7E089DDA63038F199DE52
:103320007F934BD0C0936B01D0936C01E0917A01F5
:10333000F09178010E948C3622D0C0916B01D0911F
:103340006C01E0917A01F09178010E948C367F91B6
:1033500070933801DECFA7E069DDA63038F079DE62
:103360007F9305D07F9170933801D3CFB1CE25D014
:10337000DE01A0936B01B0936C010E947A34A0919E
:103380008001B0918101C0918201D0918301219689
:10339000AC17BD0708F008951196A0938001B09373
:1033A00081010BD0E0916B01F0916C01C0936B0136
:1033B000D0936C010E948C36E2CFA0918001B09135
:1033C00081010E94AE0B00917C0111270E947D0BB0
:1033D000D0917801DB1BA0918001B09181019D9774
:1033E0009D970E94AE0B00917E0111270E947D0BDC
:1033F000C0917A01CB0F0895AF3F31F42C9A2CBCC9
:10340000ACE5ACBD3DBC0895A7F92CBCAF73A0647E
:10341000ACBD3DBCA5B1A4FBA5B90895BDB5B7FF32
:10342000FDCF08955C2F4D2FCF93DF9307D0DF9111
:10343000CF9108955091720140917301433038F457
:10344000DDE0CCE3C50FD41FA991BB2710C05050BD
:10345000444058F0550F441F433038F4DDE0CCE3CE
:10346000C50FD41FA991B99102C082E1089540917E
:10347000720150917301430D521D4093720150939C
:103480007301803009F408954F914F910895A0EB96
:10349000B1E04FEF52E24D935A95E9F7C8EAD1E017
:1034A00040E25A91503211F44A95D9F7442EA0EBDC
:1034B000B1E0C8E8D1E04C0EA03D28F4C41518F4E2
:1034C0004881403009F408958AD04F3FE1F371D02C
:1034D0004F3FC9F3403081F78FD0403069F73DD07E
:1034E000403051F70AD0403039F74991413618F051
:1034F0004B3708F440524D93DFCF4881403320F0E2
:103500004A3310F4405302C044270895642F7727AC
:1035100021964881403380F04A3370F44053660F5F
:10352000771F0B01660F771F660F771F600D711DE8
:10353000640F721D2196EDCF703029F04DE14D934F
:103540007D936D9308956A3020F04CE14D936D9317
:103550000895605D6D934CE108954881443211F007
:103560004427089566277727219658815033B0F075
:103570005A3310F4505308C05A3508F050525134A1
:1035800068F0573458F457535F70529544E0550F24
:10359000661F771F4A95D9F72196E7CF703029F03B
:1035A0004FE14D937D936D9308954EE14D936D934F
:1035B00008954881423211F04427089521964D9391
:1035C0004991423219F44D9341E00895403029F475
:1035D00042E24D934FEF4D9308954D93F1CF4881C3
:1035E000473211F04427089521964D934991403078
:1035F000E1F74FEF4D930895FF93EF93BF93AF9390
:103600005F93ECE9FBE40E014591403089F068944A
:1036100057E0A591AE3239F0B991B13608F0B05209
:10362000AB1709F0E8945A95A1F716F0E001EBCF3B
:103630005F91AF91BF91EF91FF91403041F04D9379
:103640004F934881403211F42196FBCF4F9108955A
:10365000CBE8D1E0A0EBB1E040E2E0E24993EA95AB
:10366000E9F7A097A03D29F04D91423010F04F3F6F
:1036700011F429920895403220F0403810F486D099
:10368000F1CF4C3121F4ED91FF2719D0EBCF4D3123
:1036900021F4FD91ED9113D0E5CF4E3131F444E2A8
:1036A00075D0ED91689449D0DDCF4F3131F444E2CB
:1036B0006DD0FD91ED9134D0D5CF50D0D3CFE894DB
:1036C0004FE24395E051F742E0F7E05FF84D4033B9
:1036D00011F063D068944FE24395E85EF340E0F761
:1036E000E851FC4F16F0403311F057D068944FE288
:1036F0004395E456F040E0F7EC59FF4F16F04033A5
:1037000011F04BD068944FE24395EA50E8F7E65F3A
:1037100016F0403309F041D040E34E0F3ED00895FB
:10372000E8944F2F42954F7011F012D068944F2FAC
:103730004F700EF011F00CD068944E2F42954F70E0
:103740000EF011F005D068944E2F4F7001D00895FF
:10375000405D4A3308F0495F20D00895ECE9FBE46E
:103760005591503009F40895451711F03796F8CF68
:103770005F9357E045914E3209F00FD05A95D1F73B
:103780005F915C3110F040E208D008954993CB3A44
:1037900018F029924F914F9108954993CB3AE0F355
:1037A00029924F914F91F6CFA0914A01A0936E01BB
:1037B000AA270E944231A0913801A0936A01A091EA
:1037C0001B01A0936D01A0913601A0936901209285
:1037D0003601E8EDF1E0CCE3D7E0BEE2AEE14191A5
:1037E0004993AA95E1F7BA95C9F70895A0916E019A
:1037F0000E944231A0916D01A0931B01A0916A012A
:10380000A0933801A0916901A0933601ECE3F7E0A1
:10381000C8EDD1E0E2CFC6E1D4E0E8ECF6E041B19A
:1038200050B168E0A9E4BFEA469510F4AFE4BFE206
:10383000A993B193A0E3B0E8569510F4A1E3BEE4D8
:10384000AD8FB58F6A9571F70895452FA6E10E9457
:10385000B1314F5B0E94BC324DE30E94BC32A7E104
:103860000E94B131C0EADCE0C50FD21DC50FD21DE8
:10387000A991B9919DE00E94D9310895A3E10E94D8
:103880006734A5E0C62FCA95AC9FCCEFDCE0C00D35
:10389000D11DA881A7FF09C00E944E34FF43414CAF
:1038A0004C202000A981AF770DC00E944E34FF4606
:1038B0004F5220004A8146954F5B0E94BC320E94C5
:1038C000BB32A981BB27A39592E00E94D9314AE37C
:1038D0000E94BC32BB27A881AF770E94D9310895DE
:1038E00020921B019927A7E00E94B1310E94493222
:1038F0000E944E3412004249542030313233343564
:10390000363700000E944E341300444952000E9492
:103910004E3414004C455600EAEFFBE30E94E638B3
:10392000A5E00E94B1310E944E3400004156522D54
:1039300043686970426173696332204D4F4E2020A5
:1039400020205000409143014F5C0E94BC320E94F5
:103950004E34FF3A000092E0BB27AC2DA3950E94A5
:10396000D9310E944E34FF3A0000BB27AD2DA395FC
:103970000E94D931EBE8F1E0C6EFD1E0AEE141EFD2
:10398000B191B03031F0BE8F4CAF4993AA95C1F7D9
:1039900006C0B0E2BE8F4CAF4993AA95D1F7A7E11C
:1039A0000E94B131C0E0D4E0E1E1F0E10E948D3548
:1039B0009DE050E0452F4C5FB42FAA270E9467344A
:1039C00044DF53955D30B1F7452F4950B42FA9E03E
:1039D0000E9467343ADF53955A31B1F7A7E30E944A
:1039E000B131C3E1D4E0EDE1F0E10E948D350E94F8
:1039F0004E340413535441434B3A00009927BB27DC
:103A0000A09170010E94D9316CE0C0917001C6177D
:103A100020F0C61BB4E0B60F31DF6A95B1F7089508
:103A20004F935F936F937F93EF93FF93CF93DF93C6
:103A3000AF93BF93AF92BF928F939F93B5DE08DE93
:103A40004FDF31D08827A09139014D3E11F4A1609C
:103A500014C0413F11F4AA2710C0423F11F4A460E2
:103A60000CC0433F39F4C2DE0E94EA36AA270E9406
:103A70004231E6CF443F29F71FC0A093390140915E
:103A800022014030E1F7B2DE9F918F91BF90AF905D
:103A9000BF91AF91DF91CF91FF91EF917F916F91A6
:103AA0005F914F91089520922301B5DE409123014B
:103AB0004030D9F30C9497370E94F13670E04424DB
:103AC00025D0ECEDFBE30E94E6380E94EA364D3E3D
:103AD00011F4A160D2CF443F19F40E94F136B0CF67
:103AE000463E31F4703069F37A950E94F136E8CFA2
:103AF000473E31F47A3028F773950E94F136E0CFD3
:103B0000433FF9F643940E94F136DACFA7E00E94D2
:103B1000B1310E9449320E944E3400004156522D6C
:103B200043686970426173696332204172726179DE
:103B3000205669657700A0E60E94B1310E944E349C
:103B40000200416472202000A0E50E94B1310E9471
:103B50004E340205202020202020202020446174A3
:103B6000612020202020202020202020000060E450
:103B7000679FCCE3DDE0C00DD11DF00163E0A0E064
:103B8000B62F0E946734A6E00E94B131DF0191E0B8
:103B90000E943432A5E0B62F0E946734A5E00E944F
:103BA000B13190E058E0A991B0E00E943432442D48
:103BB00040FF0BC0A7E10E94B131219749910E94BB
:103BC000BC32A5E00E94B13102C00E94BB325A95BE
:103BD00051F738966395633191F6089520457869D9
:103BE000742020202020202020202020202020435E
:103BF00068617220204D6F6E202020457869742006
:103C00002020476F2020205374657020205669655E
:103C100077202041727261792092360120924A0108
:103C2000A5E00E94B131C0E0D0E0EDE1F6E10E94F4
:103C30002936A0E50E94B1310E944E34010244466B
:103C40004C4153482073697A653A20000E94D32280
:103C50004F3749F40E944E34FF353132204B6942D0
:103C60007974650011C04F3F41F40E944E34FF311A
:103C7000204D69427974650007C00E944E34FF30C0
:103C800020427974650013C00E94C4224130D1F0F3
:103C9000E4EBFEE3E8940E949338413009F434C029
:103CA000453009F4B9CF423099F733D0B5CFE0EFC2
:103CB000FEE3E8940E949338413009F425C0453072
:103CC000B1F7AACFE8E7FEE3E8940E9493384130C9
:103CD00009F41AC0473019F40E94961F9DCF4A304C
:103CE00011F417D099CF423011F46DD095CF4330F5
:103CF00019F40E94EF1F90CF443019F40E94432022
:103D00008BCF4530F9F688CFA0912201A030E1F7A2
:103D100008950E949D3B4F466F726D6174204D6502
:103D20006469756D3F00413009F00895A6E20E9474
:103D3000B131C2E0D8E0EBE1FCE00E94FA350E942C
:103D40004E340903466F726D617474696E672E2E6E
:103D50002E202020202020000E944E340B03000043
:103D60000E94D622803001F50E944E340903466F2E
:103D7000726D617474696E672E2E2E20446F6E65AD
:103D80002100A2E70E94B1310E944E340B03202093
:103D900020507265737320616E79206B65792120E4
:103DA00020000E94EA3608950E944E340903466FAF
:103DB000726D617474696E672E2E2E204572726F5B
:103DC00072210000DECFA0E60E94B131C4E0D8E04D
:103DD000E9E1FDE00E94FA350E944E340905417682
:103DE00061696C61626C653A00000E944E340A059C
:103DF00046696C65733A20009CE00E94B622DF930E
:103E0000CF93DF010E94D9310E944E34FF202F0052
:103E10000E94D322A42FB0E011960E94D9310E94B3
:103E20004E340B05426C6F636B733A00AF91BF91D8
:103E30000E94D9310E944E34FF202F000E94BE22E2
:103E4000A0EFA49FD0011197B03009F413970E94FE
:103E5000D931A6E00E94B1310E944E340C052020D9
:103E600020507265737320616E79206B6579212013
:103E700020000E94EA360895204578697420204980
:103E80006E666F204261636B7570526573746F72FA
:103E900052657363616E20202020202044656C658C
:103EA0007465202020202020202020202020466F04
:103EB000726D6174204578697420466F726D61740B
:103EC00020202020202020202020202052657363E5
:103ED000616E202020202020202020202020202053
:103EE00020202020202020202020202020202020D2
:103EF00020457869742020202020202020202020A8
:103F0000202020202020202052657363616E202015
:103F100020202020202020202020202020202020A1
:103F200020202020202020202020202077270FD193
:103F3000A4E00E94B131C1E0D2E0ECE1F5E10E94E1
:103F40002936A0E40E94B1310E944E340302446538
:103F50006C6574652066696C6500B4D070937801F7
:103F600008D34C3FD1F350D1413019F4A72FC3D21D
:103F700011D308957727EBD0A4E00E94B131C1E0BE
:103F8000D2E0ECE1F5E10E942936A0E40E94B131D3
:103F9000A0E1A0937C010E944E3403025361766538
:103FA00020500000CAD28ED070937801E2D2403EF9
:103FB00030F4403171F0483161F0F6D0DCCFD6D228
:103FC000D03021F4CC3010F429D1D5CF94D2B6D151
:103FD00008950ED1413079F68ED2BCD1089577275D
:103FE000B6D0A4E00E94B131C1E0D2E0ECE1F5E14D
:103FF0000E942936A0E40E94B131A2E1A0937C0185
:104000000E944E3403024261636B757000005AD007
:1040100070937801AED2403920F4423161F0C4D0BF
:10402000DFCFA4D2D03021F4C03610F4F7D0D8CFEF
:1040300062D226D20895DCD0413091F65CD22CD2E7
:104040000895772784D0A4E00E94B131C1E0D2E086
:10405000ECE1F5E10E942936A0E40E94B1310E9412
:104060004E3403024C6F61642050000066D22AD0A7
:10407000709378017ED2403121F0483111F0A2D006
:10408000E1CF90D10895772762D0A4E00E94B131AA
:10409000C1E0D2E0ECE1F6E10E942936A0E40E9402
:1040A000B1310E944E340302526573746F72650021
:1040B00009D0709378015DD2423111F08ED0E4CFF7
:1040C00003D208957727B5D00BD10E94EA364D3E32
:1040D00021F42FD14F914F9108954A3E09F408954C
:1040E000403E19F40FD17727EECF413E21F40AD19B
:1040F00070918001E8CF443E49F4703031F302D131
:104100007150472F4F704F30F1F2DECF453E59F4DA
:1041100040918001471709F4D8CFF4D07395472F09
:104120004F7089F2D1CF463E29F4703170F2EAD057
:104130007051C9CF473E51F4409180014F3031F06A
:104140004051471718F0DED0705FBDCFBECF0E9440
:10415000D322403019F44F914F911BC040938001FE
:104160000E94C1360E94C1360FD2413019F04F91E2
:104170004F9101C008950E94743B4F44464C4153F7
:1041800048206E6F7420666F726D61747465640090
:1041900008950E94743B4F44464C41534820657239
:1041A000726F7221000008950E94743B4F43616E4C
:1041B000206E6F742073617665206F6E207468695D
:1041C000730008950E94743B4F4E6F204241534943
:1041D000432066696C65000008950E94743B4F4E51
:1041E0006F204241434B55502066696C650008952D
:1041F0000E949D3BC04F7665727772697465206638
:10420000696C653F000008950E949D3B4F44656CBA
:104210006574652066696C653F0008950E94743B73
:104220004F4E6F207370616365206C65667400008B
:1042300008955F936F937F93A72FA07FA0936C0146
:10424000A0916C01AF70AB5FBA2FA4E00E946734FD
:10425000A6E00E94B131A0916C01BB2795E00E94BD
:10426000D9310E94BB32A5E00E94B131A0916C010E
:10427000A09378017ED1B5D04F3F61F1A0916C0140
:10428000A093780140E040937A0142E040937C01A2
:10429000882783D1803091F4CCE3DFE00E94BB32E9
:1042A0005CE05F934991403808F04EE2403208F4F8
:1042B00040E20E94BC325F915A9599F7A0916C013F
:1042C000A395A0936C01AF7009F0BACF7F916F9165
:1042D0005F9108955DE00E94BB325A95E1F7EECF01
:1042E0004F935F93C4E2D5E0472F4F705EE1459F47
:1042F000C00DD11D52EF47E159934A95E9F75F91FF
:104300004F9108954F935F93C4E2D5E0472F4F70CC
:104310005EE1459FC00DD11D5CE044E059934A9594
:10432000E9F75AE043E159934A95E9F75F914F91D4
:104330000895A0912201A030E1F7089570937801CB
:104340004CE040937A0140E140937C0120D18030E1
:1043500009F01FCF7093780190914901ECE0F0E9EA
:104360009770929540EC949FE00DF11D04913C975D
:1043700040E10E3409F448E10E94C83E40E04F930A
:1043800000E0CCE3DFE0159119930A95E1F7409343
:104390007A0142E040937C0103D14F9143954C3028
:1043A00071F70895909149019770E0E0F0E99295D6
:1043B00040EC949FE00DF11D40E04F9340937A0153
:1043C00042E040937C0170937801E7D0CCE3DFE0DA
:1043D0000E94677932964F9143954C3071F77894EB
:1043E0000895403139F40E944E34FF4241533A005F
:1043F00040E10895423139F40E944E34FF42555055
:104400003A0042E10895443139F40E944E34FF5598
:1044100053523A0044E10895463139F40E944E3433
:10442000FF4348383A0046E10895483139F40E9484
:104430004E34FF42494E3A0048E108954A3139F47A
:104440000E944E34FF47504F3A004AE108954C31E4
:1044500039F40E944E34FF53414D3A004CE1089527
:104460004E3139F40E944E34FF4C424C3A004EE13A
:1044700008950E944E34FF2D2D2D2D004FEF0895ED
:104480007093780140E640937A0142E140937C01C9
:104490007ED0803009F07DCE709378014427E0E033
:1044A000F0E94F93CCE3DFE00024159019920A94D1
:1044B000E1F740937A0142E040937C0171D04F9143
:1044C0004395403671F7089540E0E0E0F0E94F93FE
:1044D00040937A0142E040937C01709378015DD073
:1044E000CCE3DFE00E94677932964F9143954036E6
:1044F00071F7789408950E9424014F9340913801F8
:10450000409381014CE440933801C6E0DAE0E7E1F2
:10451000FCE00E94FA350E944E340B075772697412
:10452000696E6720646174612E2E2E0040918101B6
:10453000409338014F910C941D01CAE3CAE34091A6
:104540004901942F4F5C499340E249934BE54993CD
:10455000409135014F934068409335010E9499790D
:104560004DE549934F914093350108950E942E40A7
:1045700008950E94F6400E94CC3E08950E94753E28
:1045800008950E94FA3E08950E940D4008950E94E9
:104590008B4008950E94FE4008950E947441089542
:1045A0000E941A4108950E94833E08950E94A73FE9
:1045B0000895A1E00E944B382092360120924A01D2
:1045C000A7E00E94B131C0E0D0E0EDE1F6E10E9449
:1045D0002936A0E70E94B1310E944E3401024156B3
:1045E000522D4368697042617369633220636F6E54
:1045F0006669677061676500A7E00E94B1310E943B
:104600004E341401436865636B73756D3A20000086
:104610006AD168D0ECE1F9E4E8940E949338413023
:1046200011F40C940000423059F44091180150E20A
:104630004527409318010E9407790E946E24E9CF14
:10464000433071F440911801542F53955170487FB5
:10465000452B409318010E9407790E946E24D9CF00
:10466000443059F44091180150E145274093180116
:104670000E9407790E946E24CCCF453059F44091B6
:10468000180158E04527409318010E9407790E94BD
:104690006E24BFCF473049F440916501542F4395B4
:1046A0004770587F40936501F0CF483051F44091F6
:1046B0001801405C409318010E9407790E946E2403
:1046C000A8CF493051F440916501405840936501AD
:1046D0000E9407790E946E249CCF4A3011F40E94F8
:1046E000E42D67CFA6E00E94B1310E944E34030151
:1046F0004B6579626F617264206C61796F75743A91
:1047000000000E944E34050153657269616C20738C
:10471000706565643A000E944E34070149324320B7
:1047200073706565643A00000E944E34090153506D
:10473000492073706565643A00000E944E340B0195
:10474000454550524F4D20616464726573733A0061
:104750000E944E340D014C696E6520456E643A002E
:104760000E944E340F0153657269616C20696E744A
:104770006572666163653A00A1E70E94B13170918C
:10478000180175FD0AC00E944E34031244452028CA
:1047900051574552545A290009C00E944E34031201
:1047A00055532028515745525459290070FD0AC0CD
:1047B0000E944E3405122031323030204270732076
:1047C000200009C00E944E340512203234303020BF
:1047D00042707320200074FD0AC00E944E340712FC
:1047E0002020313030206B487A20200009C00E9400
:1047F0004E3407122020343030206B487A202000BD
:1048000073FD0AC00E944E3409122020202035205A
:104810004D487A20200009C00E944E340912202001
:10482000313536206B487A202000707C51F40E948C
:104830004E340D122020206E6F6E65202020200047
:1048400021C0703851F40E944E340D12206F6E6CEE
:1048500079204C462020200015C0703451F40E946D
:104860004E340D12206F6E6C7920435220202000B0
:1048700009C00E944E340D12202043522B4C46207A
:10488000202020007091650177FD0AC00E944E34FF
:104890000F12202073696D706C652020200009C004
:1048A0000E944E340F12207374616E646172642032
:1048B00020000E944E340B12202020202000472F81
:1048C0004770405D0E94BC320E944E34FF20202081
:1048D00020200000A7E00E94B1310895A09122019C
:1048E000A030E1F70895AA27CC27DD27EE27FF2780
:1048F0001590C10DD21DA21DFE38D1F7EE27F0EFA5
:104900001590C10DD21DA21DF030D1F7BB279FE03D
:104910000E943432DE010E943432089520457869C5
:104920007420204B65796220205365722020204935
:1049300032432020205350492020202020202020B6
:10494000454550524F4D204C696E65205365726944
:104950006E7420436C6F6E65AEE0A0933801C1E0C9
:10496000D4E0ECE1F2E10E94FA350E944E340505F4
:1049700000000E9479020E944E340603202020206D
:104980002028632920323030362D32303039202033
:104990002020202000000E944E34070320202020E9
:1049A0006279204A6F65726720576F6C6672616D1D
:1049B000202020200000A2EAA09338010E944E345B
:1049C0000903202020202020446564696361746508
:1049D0006420746F20202020202000000E944E348C
:1049E0000A03466C6F7269616E2C204572696B20F8
:1049F000616E64204469616E612E0000AEE0A09398
:104A000038010E944E340C025468697320736F663B
:104A10007477617265206973206C6963656E736574
:104A200064000E944E340D04756E646572207468D3
:104A300065207465726D73206F6620746865200050
:104A40000E944E340E04474E55205055424C494367
:104A5000204C4943454E534520562E3320000E949A
:104A60004E340F0355736520697420617420796F8B
:104A70007572206F776E207269736B210000A2EC53
:104A8000A09338010E944E341107205052455353D1
:104A900020414E59204B455920000E94EA36089586
:104AA00061E00E947C38509122015D3E09F4089536
:104AB0004531B1F790914901E0E0F0E997709295A6
:104AC00040EC949FE00DF11DCCE3DDE050E045911A
:104AD00049935A95E1F7CCE3DDE00E949C3D0E94AA
:104AE0007C38509122015D3E11F34630A1F7639569
:104AF000CCEBDDE00E949C3D0E947C38509122016D
:104B00005D3EA9F24630A1F763956931E9F644E0CC
:104B10000E9460380895909149019770E0E0F0E9B3
:104B2000929540EC949FE00DF11D45E10E946038A4
:104B300060E06F93CCE3DFE00E94793D803041F08C
:104B4000813051F1883241F145E10E946038F2CF65
:104B500046E00E946038CCEBDFE00E94793D803077
:104B600041F08130C9F08832B9F045E10E946038E7
:104B7000F2CF0E9467797894329646E00E946038BE
:104B80006F9163956C30A9F60E946C384430E1F760
:104B900046E00E94603808956F91089502414253A3
:104BA000282E2E2E0353474E282E2E2E04535152BC
:104BB000282E2E2E054E4F54282E2E2E06524E44B1
:104BC000282E2E2E07414443282E2E2E08494E28EB
:104BD0002E2E2E2E09585045454B282E0A54454D51
:104BE00050282E2E0B4C4F282E2E2E2E0C484928A6
:104BF0002E2E2E2E0D4B4559282E2E2E0E4550456D
:104C0000454B282E0F455252282E2E2E1041522849
:104C10002E2E2E2E1153494E282E2E2E12434F5338
:104C2000282E2E2E134654595045282E14465349EB
:104C30005A45282E155053544154282E1653504986
:104C4000282E2E2E174D454E55282E2E18564259D9
:104C50005445282E1958524543282E2E1A464649A7
:104C60004E44282E1B44424954282E2E805052492F
:104C70004E542E2E81434C532E2E2E2E82474F54AF
:104C80004F2E2E2E83424F582E2E2E2E8441434FD0
:104C900050592E2E8553594E432E2E2E86454E4466
:104CA0002E2E2E2E8742434F50592E2E8854484583
:104CB0004E2E2E2E89504F532E2E2E2E8A4E4F546E
:104CC000452E2E2E8B4F4E53594E432E8C5252450D
:104CD00041442E2E8D5257524954452E8E474F53E4
:104CE00055422E2E8F52455455524E2E90564D4FB2
:104CF00044452E2E914E4558542E2E2E92494E50FC
:104D000055542E2E93504C4F542E2E2E94574149CD
:104D1000542E2E2E95545345542E2E2E96544745E0
:104D2000542E2E2E974653454C454354984F4E458E
:104D300052522E2E99535055542E2E2E9A5347458B
:104D4000542E2E2E9B45504F4B452E2E9C4745549E
:104D50005049582E9D434952434C452E9E434F4C3B
:104D60004F522E2E9F424F524445522EA0464F4E38
:104D7000542E2E2EA150554D502E2E2EA258504F4F
:104D80004B452E2EA356504F4B452E2EA44C494D2D
:104D900049542E2EA547455443484152A6445241FA
:104DA00057544F2EA7504C41592E2E2EA8535052D7
:104DB0004954452EA95343524F4C4C2EAA425245BA
:104DC000414B2E2EAB464153542E2E2EAC534C4FFE
:104DD000572E2E2EAD445241572E2E2EAE49434F04
:104DE0004D4D2E2EAF444154412E2E2EB0435445EE
:104DF00058542E2EB146524541442E2EB24657529B
:104E00004954452EB343424F582E2E2EB447455495
:104E100041545452B54644454C455445B646424F1C
:104E2000582E2E2EB750414C45545445B8464F523B
:104E30002E2E2E2EB949462E2E2E2E2EBA444952F3
:104E40002E2E2E2EBB4F55542E2E2E2EBC464349B1
:104E500052434C45BD414C4552542E2EBE46435202
:104E600045415445BF41534B2E2E2E2ECE474F5316
:104E70002E2E2E2EC03F2E2E2E2E2E2EC1585345B6
:104E80004E442E2EC2474F2E2E2E2E2EC3544F2E62
:104E90002E2E2E2EC44C4F4144502E2EC643434836
:104EA00041522E2EC742432E2E2E2E2EC85341562F
:104EB00045502E2EC94152432E2E2E2ECA4E4F2E15
:104EC0002E2E2E2ECB5049452E2E2E2ECC52524415
:104ED0002E2E2E2ECD5257522E2E2E2ECF524554E0
:104EE0002E2E2E2ED0564D2E2E2E2E2ED2494E50F8
:104EF0002E2E2E2ED3504C2E2E2E2E2ED7465345F0
:104F00004C2E2E2EDC4750582E2E2E2EDD43492EB1
:104F10002E2E2E2EDE434F4C2E2E2E2EDF424F2EC7
:104F20002E2E2E2EE258502E2E2E2E2EE356502EA2
:104F30002E2E2E2EE44C494D2E2E2E2EE547434884
:104F40002E2E2E2EE644544F2E2E2E2EE853505247
:104F50002E2E2E2EED44522E2E2E2E2EEE49432E88
:104F60002E2E2E2EEF44412E2E2E2E2EF146524462
:104F70002E2E2E2EF24657522E2E2E2EF447415410
:104F80002E2E2E2EF54644454C2E2E2EF750414CFB
:104F90002E2E2E2EFC4643492E2E2E2EFE464352FA
:104FA0002E2E2E2E002E2E2E2E2E2E2EA0911401C1
:104FB000B0911501ED01E2EBF2E0CE0FDF1FF6EF4D
:104FC000E0911A01FE0F7F934F92EEE14E2E699110
:104FD000ED915491762F7295762757FD672768B922
:104FE000ED91000056FD76B9049055FD76B96991B2
:104FF000162E54FD76B91294162653FD76B907FC89
:1050000061254A9452FD76B9502D712D41F760917A
:105010001B0168B94F907F91EE91F0911A01F395C1
:10502000FA3029F4FF27A0931401B0931501F093EF
:105030001A010C943F30A0911401B0911501F82D84
:10504000FA95CCE5DBE0F295FF70E5E1EF9FC00D4E
:10505000D11D10901B01FD916991462FF0FD4295E5
:1050600048B9562F452FF1FD429548B90000452F0C
:10507000F2FD429548B96991452FF3FD429548B933
:105080000000452FF4FD429548B90D90452FF5FDE0
:10509000429548B90000452FF6FD429548B9F7FD05
:1050A0005295462F00FC429558B9F02DEA95C1F66D
:1050B00018B8EE91F0911A01F395F23029F4FF2718
:1050C000A0931401B0931501F0931A010C943F3092
:1050D000A0911401B0911501D1E0FEE110901B01E7
:1050E000ED91CE2FC370588158B9CE2FC695C69575
:1050F000C3705881E29558B9CE2FC3705881CE2F16
:10510000C69558B9C695C3705881ED91CE2F58B940
:10511000C3705881FA9541F718B8EE91F0911A01D1
:10512000F395F33029F4FF27A0931401B0931501F0
:10513000F0931A010C943F30A0911401B091150125
:105140000F9310901B01EAE2D1E0CD91C6950C2F90
:10515000C295CF70F881F8B9C02F0000CF70F881E8
:10516000000000000000F8B9CD91C6950C2FC29543
:10517000CF70F881EA9579F718B811970F91F091EF
:105180001A01F395F43029F4FF27A0931401B0938A
:105190001501F0931A010C943F30A0911401B091C5
:1051A0001501D0910001C0910101C295DC0FDE7E96
:1051B000E0E110901B01FD914D2FF0FD429548B9A3
:1051C0000000000000004D2FF1FD429548B900009D
:1051D000000000004D2FF2FD429548B9000000008C
:1051E0004D2FF3FD4295000048B9000000006D2FDF
:1051F0004D2FF4FD429548B90000CD91F5FD629523
:105200005D2F68B900000000F6FD52956D2F4D2FFF
:1052100058B9F7FD6295C0FD42950000000068B9DD
:10522000FC2F00000000EA9551F6000018B8EE913E
:10523000F0911A01F395F33029F4FF27A09314019C
:10524000B0931501F0931A010C943F30A091140112
:10525000B0911501C0914D01D82DF6EFE0911A01E2
:10526000FE0FE395E0931A01EA3088F1EC3069F51E
:105270009396A0931401B093150120921A01DC308B
:1052800031F4D0914C01D0934D010C943F30D83182
:1052900089F4A1E4B2E0C0913A01D3E2CD9FA00D20
:1052A000B11DCFE0A0931401B0931501C0934D013F
:1052B0000C943F30D83D49F4CBE4AEE1B2E0A0938A
:1052C0001401B0931501C0934D010C943F300F931E
:1052D0001F932F93D83D28F4DC2F0C2F1C2F2C2F3D
:1052E00005C029E61DE208E8DCECCBE46C2F7C2F3E
:1052F0007295ED91E7FD6727EF775491ED9168B9CD
:10530000172E56FD16B86C2F7C2F729555FD16B8CA
:10531000E7FD672754FD16B8EF77000053FD16B878
:10532000049052FD16B8502DED9168B9172E56FD18
:1053300016B86C2F7C2F729555FD16B8E7FD6727C0
:1053400054FD16B8EF77000053FD16B8049052FDD7
:1053500016B8502DED9168B9172E56FD16B86C2F62
:105360007C2F729555FD16B8E7FD672754FD16B8DA
:10537000EF77000053FD16B8049052FD16B8502D7B
:10538000ED9168B9172E56FD16B86C2F7C2F7295CB
:1053900055FD16B8E7FD672754FD16B8EF770000F6
:1053A00053FD16B8049052FD16B8502DED9168B912
:1053B000172E56FD16B86C2F7C2F729555FD16B81A
:1053C000E7FD672754FD16B8EF77000053FD16B8C8
:1053D000049052FD16B8502DED9168B9172E56FD68
:1053E00016B86C2F7C2F729555FD16B8E7FD672710
:1053F00054FD16B8EF77000053FD16B8049052FD27
:1054000016B8502DED9168B9172E56FD16B86D2FB0
:105410007D2F729555FD16B8E7FD672754FD16B828
:10542000EF77000053FD16B8049052FD16B8502DCA
:10543000ED9168B9172E56FD16B86D2F7D2F729518
:1054400055FD16B8E7FD672754FD16B8EF77000045
:1054500053FD16B8049052FD16B8502DED9168B961
:10546000172E56FD16B86D2F7D2F729555FD16B867
:10547000E7FD672754FD16B8EF77000053FD16B817
:10548000049052FD16B8502DED9168B9172E56FDB7
:1054900016B86D2F7D2F729555FD16B8E7FD67275D
:1054A00054FD16B8EF77000053FD16B8049052FD76
:1054B00016B8502DED9168B9172E56FD16B86D2F00
:1054C0007D2F729555FD16B8E7FD672754FD16B878
:1054D000EF77000053FD16B8049052FD16B8502D1A
:1054E000ED9168B9172E56FD16B86D2F7D2F729568
:1054F00055FD16B8E7FD672754FD16B8EF77000095
:1055000053FD16B8049052FD16B8502DED9168B9B0
:10551000172E56FD16B86D2F7D2F729555FD16B8B6
:10552000E7FD672754FD16B8EF77000053FD16B866
:10553000049052FD16B8502DED9168B9172E56FD06
:1055400016B8602F702F729555FD16B8E7FD6727C6
:1055500054FD16B8EF77000053FD16B8049052FDC5
:1055600016B8502DED9168B9172E56FD16B8602F5C
:10557000702F729555FD16B8E7FD672754FD16B8D4
:10558000EF77000053FD16B8049052FD16B8502D69
:10559000ED9168B9172E56FD16B8602F702F7295D1
:1055A00055FD16B8E7FD672754FD16B8EF770000E4
:1055B00053FD16B8049052FD16B8502DED9168B900
:1055C000172E56FD16B8602F702F729555FD16B820
:1055D000E7FD672754FD16B8EF77000053FD16B8B6
:1055E000049052FD16B8502DED9168B9172E56FD56
:1055F00016B8602F702F729555FD16B8E7FD672716
:1056000054FD16B8EF77000053FD16B8049052FD14
:1056100016B8502DED9168B9172E56FD16B8602FAB
:10562000702F729555FD16B8E7FD672754FD16B823
:10563000EF77000053FD16B8049052FD16B8502DB8
:10564000ED9168B9172E56FD16B8612F712F72951E
:1056500055FD16B8E7FD672754FD16B8EF77000033
:1056600053FD16B8049052FD16B8502DED9168B94F
:10567000172E56FD16B8612F712F729555FD16B86D
:10568000E7FD672754FD16B8EF77000053FD16B805
:10569000049052FD16B8502DED9168B9172E56FDA5
:1056A00016B8612F712F729555FD16B8E7FD672763
:1056B00054FD16B8EF77000053FD16B8049052FD64
:1056C00016B8502DED9168B9172E56FD16B8612FFA
:1056D000712F729555FD16B8E7FD672754FD16B872
:1056E000EF77000053FD16B8049052FD16B8502D08
:1056F000ED9168B9172E56FD16B8612F712F72956E
:1057000055FD16B8E7FD672754FD16B8EF77000082
:1057100053FD16B8049052FD16B8502DED9168B99E
:10572000172E56FD16B8612F712F729555FD16B8BC
:10573000E7FD672754FD16B8EF77000053FD16B854
:10574000049052FD16B8502DED9168B9172E56FDF4
:1057500016B8612F712F729555FD16B8E7FD6727B2
:1057600054FD16B8EF77000053FD16B8049052FDB3
:1057700016B8502DED9168B9172E56FD16B8612F49
:10578000712F729555FD16B8E7FD672754FD16B8C1
:10579000EF77000053FD16B8049052FD16B8502D57
:1057A000ED9168B9172E56FD16B8622F722F7295BB
:1057B00055FD16B8E7FD672754FD16B8EF770000D2
:1057C00053FD16B8049052FD16B8502DED9168B9EE
:1057D000172E56FD16B8622F722F729555FD16B80A
:1057E000E7FD672754FD16B8EF77000053FD16B8A4
:1057F000049052FD16B8502DED9168B9172E56FD44
:1058000016B8622F722F729555FD16B8E7FD6727FF
:1058100054FD16B8EF77000053FD16B8049052FD02
:1058200016B8502DED9168B9172E56FD16B8622F97
:10583000722F729555FD16B8E7FD672754FD16B80F
:10584000EF77000053FD16B8049052FD16B8502DA6
:10585000ED9168B9172E56FD16B8622F722F72950A
:1058600055FD16B8E7FD672754FD16B8EF77000021
:1058700053FD16B8049052FD16B8502DED9168B93D
:10588000172E56FD16B8622F722F729555FD16B859
:10589000E7FD672754FD16B8EF77000053FD16B8F3
:1058A000049052FD16B8502DED9168B9172E56FD93
:1058B00016B8622F722F729555FD16B8E7FD67274F
:1058C00054FD16B8EF77000053FD16B8049052FD52
:1058D00016B8502DED9168B9172E56FD16B8622FE7
:1058E000722F729555FD16B8E7FD672754FD16B85F
:1058F000EF77000053FD16B8049052FD16B8502DF6
:10590000ED9128B82F911F910F910C943F30A091E9
:105910001401B0911501EAE8F4E0C0911A01D3E056
:10592000CD9FE00DF11D7F936EE17EE1CBE1D1E0F3
:105930005881507F452F4295542B588358B9529522
:105940004D914F7358B95991469F58B95295EF01EF
:10595000000058B9C00DD11D599158B952957A958A
:105960000000000058B9599149F7000058B9529504
:1059700060911B01000058B959917F9158B9529517
:10598000F0911A01F39558B90000000068B9FA3097
:1059900029F4FF27A0931401B0931501F0931A0185
:1059A0000C943F30A0911401B0911501ED01E2EB90
:1059B000F2E0CE0FDF1FF7E0E0911A01E395E0FB84
:1059C000E695FE0F7F934F92EEE14E2E6991ED9199
:1059D000E7F95081762F7295762757FD672768B9CA
:1059E000ED91E7F956FD76B90080000055FD76B9D6
:1059F0006991162E54FD76B91294162653FD76B988
:105A000007FC61254A9452FD76B9502D712D39F766
:105A100060911B0168B94F907F91EE91F0911A014E
:105A2000F395FA3029F4FF27A0931401B0931501E0
:105A3000F0931A010C943F30A8EDB1E0C4E1D2E03C
:105A400080921A010C94DF27A6EFB1E0C2E3D2E006
:105A5000425D40931A010C94DF27482D4A5008F408
:105A6000EBCF423D08F0F0CF58E14695A0E5B2E01B
:105A7000A40FB21D4C91459FA9EBB2E0A00DB11D42
:105A8000CFE94D915D91C395C41731F0000000003E
:105A90000000C215C1F792C04D9158B96D91C395E0
:105AA000C41731F00000529558B9C215C1F786C02D
:105AB0004D9168B95D91C395C41731F000006295AE
:105AC00068B9C215C1F77AC04D9158B96D91C395A7
:105AD000C41731F00000529558B9C215C1F76EC015
:105AE0004D9168B95D91C395C41731F0000062957E
:105AF00068B9C215C1F762C04D9158B96D91C3958F
:105B0000C41731F00000529558B9C215C1F756C0FC
:105B10004D9168B95D91C395C41731F0000062954D
:105B200068B9C215C1F74AC04D9158B96D91C39576
:105B3000C41731F00000529558B9C215C1F73EC0E4
:105B40004D9168B95D91C395C41731F0000062951D
:105B500068B9C215C1F732C04D9158B96D91C3955E
:105B6000C41731F00000529558B9C215C1F726C0CC
:105B70004D9168B95D91C395C41731F000006295ED
:105B800068B9C215C1F71AC04D9158B96D91C39546
:105B9000C41731F00000529558B9C215C1F70EC0B4
:105BA0000000000068B900000000C395C4170000A1
:105BB0000000629568B9C215C1F700C050911B0181
:105BC0000000000058B95BC20E949D3B6F436C6FA0
:105BD0006E652073797374656D3F2000413009F064
:105BE000089565D087D0803079F078D00E94743BDA
:105BF0004F4E6F20636F6E74726F6C6C65722066AF
:105C00006F756E64200008958DD0803069F066D085
:105C10000E94743B4F4E6F204D65676136343420CF
:105C2000666F756E64000895CDD09DD0EE27FF2776
:105C300050E060E00590B8D00590BDD06395603825
:105C4000C9F79ED05395A9F74CEA4ED040EA4CD004
:105C50004AD046EE49D00E94C1360E94C1360E9409
:105C6000C1364CEA41D048EA3FD03DD041ED3CD06E
:105C70000E94C1360E94C1360E94C1364CEA34D01F
:105C800044EA32D030D04CEF2FD00E94C1360E946F
:105C9000C1360E94C13622D00E94743B8053797372
:105CA00074656D20636C6F6E65640000089543E554
:105CB0004CBD2DBC249A2C984FEF4A95F1F72C9AA5
:105CC0004FEF4A95F1F72C984FEF4A95F1F72C9842
:105CD0004FEF4A95F1F70E94C13608952C9A4CE592
:105CE0004CBD3DBC089544274EBD4DB547FFFDCF8B
:105CF0004EB5089588274CEAF7DF43E5F5DFF3DF7B
:105D0000433509F081E0EFDF0895BF93AF934F93E0
:105D1000A42FBB270E9434320E94BB324F91AF9117
:105D2000BF910895882740E3DFDFDDDF40E0DCDF5F
:105D3000DADF4E3111F082E0089540E3D5DFD3DFA2
:105D400041E0D2DFD0DF463911F082E0089540E330
:105D5000CBDFC9DF42E0C8DFC6DF493019F04A3087
:105D600009F082E008954CEABFDF40E8BDDFBBDF09
:105D7000BADF0E94C1360E94C1360E94C136089522
:105D80004CE4B2DF452F4695AFDF452F440F440F5B
:105D9000440F440F440F440F440FA6DFA4DF0E94BA
:105DA000C1360E94C136089540E49EDF9CDF462F35
:105DB0009BDF402D99CF48E497DF95DF462F94DF96
:105DC000402D92CF0E9424014F934091380140937F
:105DD00081014CE440933801C5E0DAE0E8E1FCE001
:105DE0000E94FA350E944E340B06436C6F6E696E4A
:105DF000672053797374656D2E2E2E0040918101BA
:105E0000409338014F910C941D0128B818954F9379
:105E10005F936F93FF93EF93DF93CF93BF93AF9312
:105E20000F921F92FFB7FF9330921D01B0913D0179
:105E3000B7FF5C98B7FD5C9A4B99BE7F4B9BB160F6
:105E4000A0916501C1E0A7FDBC27B0933D01C4E16D
:105E5000D1E05F89A889E9890A881B88A00DE11D26
:105E6000A88BE98BFFA14491AD89AF73AF3309F4DF
:105E7000452F5AA54503B0E8B10DB093B300EE89A4
:105E8000FF89488D598DAA27E2FDA095E5FDA095D3
:105E9000F4FDA09557FDA095AA1FEE1FFF1F441FFC
:105EA000551FEE8BFF8B488F598F830C921CEBA9EB
:105EB000FF81EF23E8B97894E9A190FC04C0F8A52C
:105EC0008F1608F4A9C071F4409110014F3F51F0B2
:105ED000409112014A9521F4409111013092130131
:105EE00040931201FCE0E2FFFDEE8F1639F45E985C
:105EF000E3FFC5C0B2E8B0938000C1C0F1E1E2FFAA
:105F0000F3EF8F1639F45E9AE3FFB9C0B2ECB093A9
:105F10008000B5C0FBE1E2FFFFEF8F1621F4EFEF49
:105F2000E0934701ACC0F2E0E2FFF9EE8F1619F4FE
:105F300020924701A4C0F9E3E2FFF7E08F1609F0D1
:105F40009EC0A8EDA883A1E0A9832E82882499246D
:105F5000AAE0A9AFA5E0E2FFA39542E3E2FF4CE38C
:105F6000BA8DB395BA1731F4BB27EB8DFC8D319602
:105F7000EB8FFC8FBA8FE885E395E41709F4EE27E1
:105F8000E887FDE8E0E0A0912901A7FDB096AC8983
:105F9000EA0FF21DB491B21511F0A395AC8BBAA71C
:105FA000A0915C01A03009F46AC0B0915D01B39585
:105FB000B0935D01BA17C0F320925D01B091640106
:105FC000BA95B093640181F7E0915E01F0915F01B1
:105FD000C0916201D09163012196A191B191B093DA
:105FE0006401E0935E01F0935F01D4D6FD1798F051
:105FF000EC1788F0A0913F01A13029F4A2E0209293
:106000005C01A0933F01E0916001F0916101E09398
:106010005E01F0935F0133C0A0918400A63EE0F3DF
:10602000A73E00F0A83E00F0A93E00F0AA3E00F016
:10603000E5FD25C0E0913501E7FD0C942629E091AE
:106040004A01E53011F40C94CD28E03011F40C94A1
:10605000D627E13011F40C941B28E23011F40C9493
:106060006828E43011F40C94D22CE63011F40C942E
:10607000872CE73011F40C942D2D0C949C28A091C2
:106080002001A5FD27C0E091C000E7FF6BC0E091B3
:10609000C600E0937101F5EFB491B0FF36C0A7FFE1
:1060A00003C0209222015BC0E33809F4E0E1F6E886
:1060B0004091180145FDFE5FEF77A4FFA6FDF39523
:1060C000A4FFA0FDE068A1FDE068E491E093210158
:1060D000A06246C0E0912101E0932201E0932301F8
:1060E000EE3E19F4A2FD0C94EF0040913901E33625
:1060F00011F4A2FD4160E03711F4A3FD4260EC3FD2
:1061000009F44460409339012AC0E03F11F4A068CB
:1061100027C0E03E11F4A06423C0E23131F4A6FDB3
:106120001EC0A160A7FDAE7F1AC0E93521F4A260B0
:10613000A7FDAD7F14C0E43151F4A6FD04C0A460F6
:10614000A7FDAB7F0CC0A860A7FDA77F08C0E13109
:1061500021F4A061A7FDAF7E02C020922201AF71A1
:10616000A09320014091180140FD0E94A17840FFBA
:106170000E94D678FF91FFBF1F900F90AF91BF9103
:10618000CF91DF91EF91FF916F915F914F911895B2
:10619000AAEBA4B9AFEFA5B9A0EEA7B9A0E0A8B942
:1061A000A0EFAAB9AFEFABB9A6B1AF77A093350115
:1061B000B2ECB0938000B9E1B0938100F4E0A2FFAB
:1061C000F4E0F0938700FEEFA2FFF6EFF093860075
:1061D00020928900FAE5F0938800F4E0F0938B00B8
:1061E000F8EDF0938A00A6E0A0936F00A2E0A4BDB2
:1061F000A1E0A5BDA1E3A7BDA3E8A093B000A1E0E5
:10620000A093B100A0E8A093B3002092B600209222
:10621000C000A0E1A093C100A6E6A093C200ACE537
:10622000B0911801B3FDAFE5ACBDA0E0ADBDA5E1F7
:1062300098D0C4E1D1E0A8EDA993A1E0A993AEE183
:106240002992AA95E9F7AAEAA0932A01A0932C0122
:106250002092360120921901AEE3A09328010F93FA
:10626000009135010F770093350106EE07C00F93BB
:106270000091350100680093350104EE00933C0164
:106280000F910895A0934A01A03021F0A43051F459
:106290000E946B39ACE3A0935001AEE2A093510190
:1062A000A6EE44C0A13069F4A8EAA0935001A4E787
:1062B000A0935101A0E0A0930001A0EEA0930101E2
:1062C00024C0A23091F4A8E7A0935001ACE4A093BD
:1062D0005101C0E0D1E0A0E0A993A0E4A993A0EA15
:1062E000A993A0EEA993A3EE21C0A33081F4A4E565
:1062F000A0935001AAE3A0935101C0E0D1E0AA27E6
:10630000B0E1A993A05EBA95E1F7A7EE0FC0A53062
:1063100081F4A0E8A0935001A0E4A0935101A0E271
:10632000A0930001A0EEA0930101A0ECA0933C017A
:106330000895A63051F4ACE3A0935001AEE2A093CF
:1063400051010E942D39A6EEF1CFACE3A09350018C
:10635000A2E0A09351010E9483390E949439A6EED5
:10636000E5CFAA0FAE7EA09338010895A295AA0F9B
:10637000A07EA0931B01089548834091350147FDFD
:1063800017C040914A01463099F0CF93DF935F9355
:106390005CE3C50FD21D473021F046E7C40F42E051
:1063A000D41F409138014E7E48835F91DF91CF9199
:1063B00008954F935F936F93AF93BF9340E2592F2C
:1063C0005370523061F0533009F44BE2B7FF05C00F
:1063D000A095B095A30DB21D4DE20E94BC32592F7D
:1063E0005C70692F6073E8944FE24395A051B74207
:1063F000E0F7A05FB84D5C3009F42BD04FE2439535
:10640000A85EB340E0F7A851BC4F53FD22D06033E3
:1064100009F4AFD04FE24395A456B209E0F7AC5966
:10642000BF4F503009F015D0603209F4A2D04FE2CE
:106430004395AA50E8F70DD0A65F603109F499D0D2
:1064400040E34A0F99D0BF91AF916F915F914F9107
:106450000895403311F068948FC091FD8DC0F6F31C
:1064600090FF089588C008954F9390FF05C04B2F6B
:10647000429509D04B2F07D04A2F429504D04A2F7E
:1064800002D04F9108954F70405D4A3308F0495F44
:1064900073C00E94240140914A01403001F1443010
:1064A000F1F0D1E0C8EDA7E1463009F0ACE5BEE17E
:1064B0002992BA95E9F7AA95D1F7413071F4A091E4
:1064C0003801AE7EDBE0CCE5B0EAA993A993BA959A
:1064D000E1F7AA24BB24209237010C941D0140E26D
:1064E000D1E0C8EDA7E1BEE14993BA95E9F7AA95D5
:1064F000D1F7409138014E7EA7E1BEE14993BA95AC
:10650000E9F7AA95D1F7E5CF20923701BF91AF9176
:106510000895AF93BF9320923701A0913601A03028
:1065200051F4A7E1AA24B394AB1571F7B6E1BB2EE1
:10653000CF93DF936CC0A13021F4BF91AF910C9445
:106540005338A23059F44DE0B0911801B6FDCAD4C9
:106550004AE0B7FDC7D4BF91AF910895A33019F4B5
:10656000BF91AF910895BF91AF915AE00E94BF3D96
:1065700008954CE201C040E2AF93BF93A091370170
:10658000A395A0933701A0913601A43030F0BF91BC
:10659000AF91542F0E94BF3D0895A030A9F0A330C1
:1065A00059F4A42FBB275F936F930E94F2176F914A
:1065B0005F91BF91AF910895BF91AF91A0913601C6
:1065C000A1FF0C9460388EC4EF93E0914A01E03053
:1065D00029F0E43019F0E63008F49AC0EF91CF9337
:1065E000DF9364D496FD35C0C7DEA395AE3131F498
:1065F000AA27B395B73111F4B6E107C0AA2EBB2E76
:10660000DF91CF91BF91AF910895AA2EBB2ED1E01B
:10661000C8ED4F93A6E1BEE14E8D4993BA95E1F7DF
:10662000AA95C9F7AEE140E24993AA95E9F7D4E00B
:10663000CAE8A6E1BEE14E8D4993BA95E1F7AA9565
:10664000C9F7AEE1409138014993AA95E9F74F9116
:10665000D7CFAB31A8F6B23198F6AD5FAA2EEF9343
:10666000FF934F925F926F927F9270F85F93E42F47
:10667000F6EFB5E04424552466245527A491A7FDE0
:10668000539550FB40F8A6FD539550FB41F8A5FDEE
:10669000539550FB50F8A4FD539550FB51F8A3FDC2
:1066A000539550FB60F8A2FD539550FB61F8F395AC
:1066B0005527A491A7FD539550FB42F8A6FD53958D
:1066C00050FB43F8A5FD539550FB52F8A4FD53959C
:1066D00050FB53F8A3FD539550FB62F8A2FD539570
:1066E00050FB63F8F395442D47DE2196452D44DE9B
:1066F0002196462D41DE6C96BA9509F0BBCF5F918D
:1067000070FA7F906F905F904F90FF91EF9178CFEC
:10671000FF93CF93DF936F937F93E42F60911901E1
:1067200060FD1EC0F6EFAA2DBB2DDAE0C49137D074
:10673000B395AA2D96FD33D096FDB395F395AA2D6A
:10674000DA95A1F7AA2DAA5F96FDAA5FAA2E7F91DE
:106750006F91DF91CF91FF91EF91BF91AF9108952C
:10676000F3E8EF77AE2FE4ECEA0FF21DAA0FEA0F81
:10677000F21DAA2DBB2DD6E0C49155D0B395AA2DFC
:1067800096FD51D096FDB395D0FD3196AA2DDA95A0
:1067900099F7AA2DAC5F96FDAC5FAA2ED8CF609179
:1067A00038016F936295C7FD629560933801A2D05E
:1067B000A39596FD9FD096FDA395C6FD6295609327
:1067C000380198D0A39596FD95D096FDA395C5FD6B
:1067D0006295609338018ED0A39596FD8BD096FD7F
:1067E000A395C4FD62956093380184D0A39596FD6E
:1067F00081D096FDA395C3FD6295609338017AD050
:10680000A39596FD77D096FDA395C2FD6295609302
:10681000380170D0A39596FD6DD096FDA3956F912C
:1068200060933801089560913801D0FDC295762FAC
:10683000C7FF7295709338015DD0A39596FD5AD02D
:1068400096FDA395762FC6FF72957093380152D0AE
:10685000A39596FD4FD096FDA395762FC5FF729513
:106860007093380147D0A39596FD44D096FDA3952B
:10687000762FC4FF7295709338013CD0A39596FD96
:1068800039D096FDA3956093380108954F934591B3
:10689000403011F44F9108956FDEF9CFFF91EF91E1
:1068A000EE0FFF1FAF93BF93B591BF3F11F0A591BE
:1068B0000ED0BF91AF914F934591403031F44F913D
:1068C0003197F695E7953196099456DEF5CFEF931B
:1068D000E0914A01E03021F0EF91AA2EBB2E0895FD
:1068E000EF91AE3108F0ADE1B73108F0B6E1AA2E74
:1068F000BB2E08950E942401C0915001CA1728F0B0
:10690000C0915101CB1708F002C00C941D014F93A8
:106910005F93C0914A01C53031F0C43041F0C3707B
:1069200039F0C23008F43FC009F47DC09AC0B1C04C
:1069300051E0AC3360F5BE3250F5B0FD550FB0FDFF
:10694000550FA0FD550FB695A695CEE1BC9FD1E0A1
:10695000C8EDCA0FD21DC00DD11DA2EBB2E0CA0F07
:10696000DB1FA881B0913801BE70B295A07EBA1726
:1069700091F0B0913801BE70AB2BAE7EA883A2EB34
:10698000B2E0CA1BDB0BB881B52BBF70B8835F9137
:106990004F910C941D01A2EBB2E0CA1BDB0BB88136
:1069A0005095B523F2CFCA2FC770C39540E0089425
:1069B000441FCA95E9F7A695A695A695EA2FC5E1C5
:1069C000F0914A01F2FDC0E1BC9FD1E0C8EDCA0FD1
:1069D000D21DC00DD11DA0913801F2FF08C0A695AF
:1069E000A170E9F44095A881A423A883D0CF5E2F9D
:1069F000B695B695B695F5E1FB9FECE5FBE0E00DAD
:106A0000F11DE50FF21DA0913801AE705081529535
:106A10005E705A1739F35081507E5A2B5083A881EB
:106A2000A42BA883B4CFCA2F509138015695537028
:106A300043E0C37031F0440F440F550F550FCA9512
:106A4000C9F74095A695A695CEE1BC9FD1E0C8EDCB
:106A5000CA0FD21DC00DD11DA881A423A52BA883C8
:106A600096CFCA2F509138015E704EE0C17011F47C
:106A7000429552954095A695CAE2BC9FD1E0C8EDDB
:106A8000CA0FD21DC00DD11DA881A423A52BA88398
:106A90007ECF51E0AC33D0F4BE32C0F4B0FD550F20
:106AA000B0FD550FA0FD550FB695A695CEE1BC9F44
:106AB000D1E0C8EDCA0FD21DC00DD11DB091380173
:106AC000B27029F0B881B52BBF70B88360CFB881A0
:106AD0005095B523F9CFCE3108F0CDE1EE3108F075
:106AE000EDE1D73108F0D6E1F73108F0F6E1EC1727
:106AF00018F40E2EEC2FC02DFD1718F40F2EFD2FBD
:106B0000D02D0895EC1718F40E2EEC2FC02DFD1784
:106B100018F40F2EFD2FD02D08950E9424015F93AD
:106B2000DADFA0914A01A030D9F4AC2FBD2FCF936A
:106B3000DF93BED1288252EBC50F52E0D51F509192
:106B400038015883DF91CF91AE1711F0A395EFCFA5
:106B5000BF1719F0AC2FB395EACF5F910C941D01CC
:106B6000A130D9F7C531C8F7E531B8F7D031A8F76A
:106B7000F03198F750913801ACE5BBE01C2F05E1EE
:106B80000D9FA00DB11DA10FB21D5D931395E117CF
:106B9000E0F7DF1711F3D395EFCF0E9424015F9345
:106BA000B1DFAC2FBD2FA6DEA395AE17E1F7A2DEB5
:106BB000B395FB17E1F79EDEAA95AC17E1F79ADED5
:106BC000BA95BD17E1F75F910C941D010E94240155
:106BD0005F9398DFBD2FAC2F8DDEAE1711F0A3951C
:106BE000FBCF88DEFB1711F0B395F5CF5F910C94C6
:106BF0001D01089592DF0E9424014F935F936BDF84
:106C00004C2FBD2FAC2F54D152EF599351EFA39578
:106C1000AE1711F05993FBCF53EF5993A42FB395AF
:106C2000BF1739F045D150EF5993AE2F41D1599349
:106C3000F5CFA42F3DD154EF599351EFA395AE1743
:106C400011F05993FBCF55EF59935F914F910C94ED
:106C50001D01D0DF5F93AF93BF93CF93DF93EF938B
:106C6000FF9339DFDE0124D15BEF59935CEEA395EE
:106C7000AE1711F05993FBCF5CEF5993FF91EF9151
:106C8000DF91CF91CF93DF93EF93FF93DE01B39525
:106C90000FD15DEF599350E2A395AE1711F05993C0
:106CA000FBCF5EEF5993FF91EF91DF91CF91CF939F
:106CB000DF93EF93FF93DE01B395AF93F9D0A2EB8F
:106CC000B2E0CA0FDB1F5091380152955E7E2196CB
:106CD000AF91A395AE1711F05993FBCFFF91EF91B0
:106CE000DF91CF91CF93DF93EF93FF93BD2FAC2F25
:106CF000BE5FDED05EEE59935DEEA395AE1711F048
:106D00005993FBCF5FEE5993FF91EF91DF91CF91B4
:106D1000BF91AF915F9108950F931F932F933F936E
:106D2000AF93BF93CF93DF93DE010FEFCE1B10F431
:106D30000195C1951FEFDF1B10F41195D195CD176B
:106D400060F000C02C2F2695D5DDAE1789F0A00F7E
:106D50002D1BD0F7B10F2C0FF7CF2D2F2695CADDA5
:106D6000BF1731F0B10F2C1BD0F7A00F2D0FF7CFAD
:106D7000DF91CF91BF91AF913F912F911F910F91D3
:106D80000895AF93A82DA73EE9F3A82DA73EE9F7F4
:106D9000AF910895EF93FF93AF93A0932901FBE880
:106DA000A6FDFCE8F0933B01AF73AA0FFDE8E0E815
:106DB000EA0FF21DA591A0932601A591A0932701AA
:106DC000209228012092240120922501AF91FF9169
:106DD000EF91089520922301409123014030E1F387
:106DE000A6C0409122014030E1F708955FD0A2EBA8
:106DF000CA0FA2E0DA1FA881BA2FAF93A171BE7E9D
:106E0000B295BA2BAF9120922301409123014030DB
:106E100041F440911C014B3110F4A883F6CFB883A4
:106E2000F4CFA88384D042C03F933DED52D020924E
:106E30002301409120014470431749F0403021F470
:106E40000E94AE07342F03C00E94CF07342F409119
:106E50002301403061F440911C014B3120F4488102
:106E60004F774883E6CF488140684883E2CF588116
:106E70005F7758833F910895D1E0C3EECA0FD21DCA
:106E80002092230140912301403061F440911C0184
:106E90004B3120F448814F774883F4CF48814068D4
:106EA0004883F0CF58815F7758830895AA2DBB2D72
:106EB000DEE1BD9FD1E0C8EDCA0FD21DC00DD11DCE
:106EC0000895F6DF0F9302EBC00F02E0D01F0F9181
:106ED0000895D3E2BD9FD2E0C4E4CA0FD21DC00D15
:106EE000D11D0895BF93BFEFB1B900001A99FECF2D
:106EF00042B9B4E6BA95F1F72998B4E6BA95F1F734
:106F0000299ABF91089545E5DBD00E945338C8ED1A
:106F1000D1E0F7E5EEE1B6D0FA95E1F7CF91DF9158
:106F2000EF91FF914F91442708954F9108954F930A
:106F30004091390141FFF9CF4D7F40933901409194
:106F40004A01463090F7FF93EF93DF93CF9344309D
:106F5000D1F2403029F44091350147FF13C025C0DC
:106F60004F9347E4ADD04F914F93405DA9D04F91DF
:106F7000413009F447C0423009F44DC0433009F4B0
:106F80005FC067C044E50E9460380E945338C8ED76
:106F9000D1E0FEE2EEE176D0FA95E1F7CF91DF9114
:106FA000EF91FF914F914427089545E40E94603886
:106FB00040914C015DD00E945338C8EDD1E0F3E020
:106FC000E3E260D00E945338FA95D1F7E3E2F09102
:106FD0003A01EF9FC00DD11DF0E1E3E248814F7708
:106FE000429549D049914F7746D0EA95B9F70E942A
:106FF0005338FA9591F7CF91DF91EF91FF914F912F
:107000004427089550D0C8EDD1E0F3E8E5E13AD047
:10701000FA95E1F7F0CF409100012AD040910101AB
:1070200027D04091020124D04091030121D03BD0D0
:10703000C8EDD1E0F4E5EEE125D0FA95E1F7DBCF3C
:1070400032D0C8EDD1E0FAE3EAE21CD0FA95E1F7DC
:10705000D2CF409100010CD04091010109D023D042
:10706000C8EDD1E0F0E4E0E10DD0FA95E1F7C3CF4F
:107070004295469547704F70405D4A3308F0495F2E
:107080000C94603848814295F6DF4991F4DFEA9527
:10709000C9F70C945338BF93B2E0A03009F0B06444
:1070A000B4BDBF910895BF934F934DE0B0911801C7
:1070B000B6FD06D04AE0B7FD03D04F91BF910895C9
:1070C000BF93B0913101B030E1F740933201BA95EE
:1070D000B0933101BF910895BF93B0913301B030A7
:1070E000E1F7BA95B0933301B0913301B030E1F7D5
:1070F00040913401BF910895BF93B0913301B030F6
:10710000E1F7BA95B0933301409122014D3E41F031
:10711000B0913301B030C1F740913401BF9108956F
:107120004BE1BF910895DF93CF93BF93AF93FF934C
:10713000EF93CEE1D7E0EEEAF1E733D0EF91FF91A4
:10714000FF93EF93F4DECCE6D4E0B0912001B2FDE2
:107150007E9616F026D001C01ED040912201A1E0FB
:107160004D3E69F0A2E0413F51F0A3E0423F39F0CB
:10717000A4E0433F21F0A5E0443F09F0DFCFB09108
:107180002001B2FDAB5F4A2FEF91FF91AF91BF910C
:10719000CF91DF910895BEE1A191A993BA95E1F74E
:1071A0000895BEE1A591A993BA95E1F708954E4ED1
:1071B0004E4E4E4EC0C0C0C0C0C080808080808017
:1071C0002E2E2E2E2E2E6E6E6E6E6E6EDF93CF9343
:1071D000BF93AF93FF93EF93CEE1D7E0EEEAF1E7F1
:1071E000E0DFEF91FF91FF93EF93CCE6D4E0D9DF9E
:1071F000CBCFACE5B0911801B3FDAFE5ACBDACE5CC
:10720000A093B800A0E0B4FDA1E0A093B900089558
:10721000FF93EF930F93E0912A01A0912B01B0917E
:107220002C01F0912D010027E2FD0095E5FD009570
:10723000A4FD0095F7FD0095001FEE1FAA1FBB1FC0
:10724000FF1FE0932A01A0932B01B0932C01F09330
:107250002D010F91EF91FF910895DF93CF93BF938D
:10726000AF93FF93EF934F935F936F937F93A8ED4B
:10727000B1E0C2EBD2E02D922197E9F740E050E077
:1072800012D043954034D9F77F916F915F914F9120
:107290007BCF67FF05C04F934C2FCD2FD42F4F913D
:1072A0007C2B660F0895E0E0F6EFF50FE40F649194
:1072B000C0913801DC2FD295C07FD07FE3E07727E3
:1072C000E8DF7295E6DF72957D93EA95C1F75395F5
:1072D0005A3049F70895DF93CF93BF93AF93FF934D
:1072E000EF934F93A0E8B7E0E0E0F6EFCAE0D0E814
:1072F00045914D93DA95E1F7F096F096B096CA95E0
:10730000B1F74F9141CFDF93CF93BF93AF93C0E5D8
:10731000D2E0A9E62992AA95E9F7ACEEB4E0399259
:1073200029921197E1F732CFDF93CF93BF93AF93B9
:10733000C8EDD1E0ACE3B0E2009038010CAEB993F7
:10734000AA95E1F723CF0E9424014F935F936F9397
:107350007F934F925F926F927F922F9320914A0179
:107360004090520150905501609054017090570127
:107370005091530160915601A22FA370E52F660F23
:10738000EE0FA33031F0660FEE0FA23011F0660F52
:10739000EE0FF62FA0915801A13071F4E20142D016
:1073A000803011F08FE133C0E3013CD0803011F028
:1073B00080E22DC060D02BC0A23091F4E20132D027
:1073C000803011F08FE123C0E3013BD0803011F019
:1073D00082E11DC0ACE3BDE06A0E7B1E70D017C019
:1073E000A33011F085E113C0A52DA33010F082E188
:1073F0000EC0ACE3BDE04A0E5B1EF20151916191FB
:10740000E30110D0803011F080E201C062D02F91F2
:107410007F906F905F904F907F916F915F914F91B0
:107420000C941D01CE0F10F48FE10895A09150012E
:10743000CA17D0F7DF0FC0F3B0915101DB17A0F7E7
:107440000895659FC00DD11D2296D33008F082E1CA
:107450000895A22F5091530160915601E52F660FB8
:10746000EE0FA33031F0660FEE0FA23011F0660F71
:10747000EE0FF62F0895571478F0D20134D0E8E7D4
:10748000F1E064D0D3012FD0E8E7F1E084D0539449
:1074900073946A9591F70895560E760E5A947A94DD
:1074A000D20121D0E8E7F1E051D0D3011CD0E8E7C8
:1074B000F1E071D05A947A946A9591F70895F301A6
:1074C00051936193D2010FD041D053946A95D1F773
:1074D0000895F20151916191D30105D05CD073946C
:1074E0006A95D1F708956F93C8EDD1E0213011F47A
:1074F00065E103C0253069F460E1B69FC00DD11D80
:107500006A2F669566956695C60FD21D4A2F6F91B4
:107510000895223069F46EE1B69FC00DD11D6A2F27
:1075200066956695C60FD21D4A2F440F6F91089538
:107530006AE2B69FC00DD11D6A2F66956695C60F8B
:10754000D21D4A2F440F440F6F9108957F936F937C
:10755000BF93AF93652F742F777029F4A991A193EE
:107560006A95E1F73FC0B0E8713019F0B6957A95A9
:10757000FBCF7727A991AB9F703019F0A291A0297A
:10758000A193119273957617A9F7A991AB9FA29138
:10759000A029A19327C07F936F93BF93AF93652FCB
:1075A000742F777029F4A191A9936A95E1F71AC015
:1075B0000F931F930FEF11E0000F110F7A95E1F772
:1075C000652F7881009570230095A191A19F072ACE
:1075D0000992712D6A95C9F768816023672B6993B9
:1075E0000F911F91AF91BF916F917F9108950E946C
:1075F00024010F931F932F9310E020E0FAE8EE2769
:10760000C0915301CF77D0915601DF7704910C9F41
:10761000A12DE0950491E0950D9FB12DA11729F4BE
:10762000B21719F4E39591F724C01A2F2B2FA091CC
:107630005201B0915501A10FB20F0E947A34A0916E
:107640005201B0915501A10FB21B0E947A34A09152
:107650005201B0915501A11BB21B0E947A34A09136
:107660005201B0915501A11BB20F0E947A34E395EB
:1076700069F62F911F910F910C941D010E94240116
:107680000F931F932F933F932FEFFAE8EE27C091AC
:107690005301CF77D0915601DF7704910C9FA12D34
:1076A000E0950491E0950D9FB12DB21721F4E3957B
:1076B000A1F73F91DECF1A2F2B2FA0915201B0914D
:1076C00055013A2FB21BA11B310F0E947A34B20F21
:1076D000B20F0E947A34B21BB21BA3953A17A8F7D7
:1076E000E395D9F63F91C5CFFF91EF91EE0FFF1FC4
:1076F0005BD03197F695E7953196EF93FF93C8E805
:10770000D1E0409138014F93FF93EF9361D00E94F5
:107710004E340B0920505245535320454E54455288
:107720002000EF91FF914F914093380153DB4A3E87
:10773000E9F757DB0E94F61B0895FF91EF91EE0FDA
:10774000FF1F32D03197F695E7953196EF93FF936F
:10775000C8E8D1E0409138014F93FF93EF9338D0C0
:107760000E944E340B08202859296573202F2028A9
:107770004E296F200000EF91FF914F914093380107
:1077800029DB493761F0493551F04E3619F04E3456
:1077900009F0F6CF26DB0E94F61B4427089521DB73
:1077A0000E94F61B41E00895C8E8D1E04591469556
:1077B0004F93477049934F9142954770499358E1D1
:1077C00045914993403011F05A95D1F72992089587
:1077D000FF93EF9392E020923601A991B991B2956F
:1077E000B077A770AB0FAA0FA0933801DF93CF93A8
:1077F0000E94D41BC2E0D8E0EBE1FCE00E94FA3525
:10780000A3E0B9E00E946734CF91DF9158E149913C
:10781000403051F0DF93CF935F930E94BC325F9171
:10782000CF91DF915A9599F7409138014295409355
:107830003801EF91FF9108950E942401C0915201F7
:10784000D09155010A8119810E3118F4173108F4CD
:1078500015D0A0915401B0915701C0915201D0911F
:107860005501B983AA83AE3138F4B73128F43CD03E
:107870007370713009F079D00C941D01C0915201E0
:10788000D09155010A8119812C813B81239F310FB1
:107890002596C00DD11DC00DD11D412FE8EDF1E0A1
:1078A0005EE1549FE00DF11DE00FF21D522F699132
:1078B00061935A95E1F74395431781F740914A0147
:1078C000463089F0412FEAE8F4E05EE1549FE00D94
:1078D000F11DE00FF21D522F699161935A95E1F766
:1078E0004395431781F70895C0915201D0915501F6
:1078F0000A8119812C813B81239F310F2596C00D70
:10790000D11DC00DD11D7727412FE8EDF1E05EE1DB
:10791000549FE00DF11DE00FF21D522F619169930C
:107920006F7009F071E05A95C9F74395431769F7ED
:10793000E0915201F09155014081742B7083409188
:107940004A01463089F0412FEAE8F4E05EE1549FB5
:10795000E00DF11DE00FF21D522F619169935A95D0
:10796000E1F74395431781F70895C0915201D091F3
:1079700055010A8119812C813B81310F2596412FB8
:10798000E8EDF1E05EE1549FE00DF11DE00FF21D26
:10799000522F699161935A95E1F74395431781F707
:1079A00040914A014630C1F0412FEAE8F4E05EE13F
:1079B000549FE00DF11DE00FF21D522F6991660FEB
:1079C00028F46E70462E6081607F642961935A9519
:1079D000A9F74395431749F708950E9424014F934F
:1079E0005F936F93E0913801437001F5A6E1B2E037
:1079F000C4E3D2E0F22D0BD0A0914A01A63031F0C1
:107A0000A8ECB4E0C6EED4E0FE2F01D06DC062E178
:107A10005AE149914D935A95E1F7149624966A9547
:107A2000B9F75AE1FD935A95E9F708954130E9F421
:107A3000ACE4B4E0CBE4D4E0F22D0BD0A0914A0149
:107A4000A43031F0AEEFB6E0CDEFD6E0FE2F01D09E
:107A50004BC063E159E14A914E935A95E1F7FE9389
:107A6000149725976A95B1F70895423001F5ACE473
:107A7000B4E0CEE2D4E0F22D0BD0A0914A01A430C4
:107A800031F0AEEFB6E0C0EED6E0FE2F01D02CC054
:107A900062E15AE14A914E935A95E1F7149724977F
:107AA0006A95B9F75AE1FE935A95E9F70895A6E168
:107AB000B2E0C7E1D2E0F22D0BD0A0914A01A43090
:107AC00031F0A8ECB4E0C9ECD4E0FE2F01D00CC03A
:107AD00063E159E149914D935A95E1F7FD9325965C
:107AE00014966A95B1F708956F915F914F910C9438
:107AF0001D014F935F937F93FFDA4B3111F481E0C7
:107B000015C04130C9F7E8DA642FE6DA409564170A
:107B100011F084E20BC070E85527DEDA540F499368
:107B20007A95D9F7D9DA451729F488277F915F919B
:107B30004F91089584E2FACF4F935F937F9341E092
:107B4000BFDA462FBDDA4095BBDA70E85527499178
:107B5000540FB6DA7A95D9F7452FB2DA7F915F9153
:107B60004F9108955E984CE54093B80044E84093E7
:107B7000BC0044E94093BC00089544EA0EC0509311
:107B8000BB0044E80AC044EC08D05091BB00089503
:107B900044E803D05091BB0008954093BC0040914D
:107BA000BC0047FFFCCF6091B900687F0895E5DF16
:107BB000683089F4572F550F5E70506AE0DF6831E6
:107BC00051F45B2FDCDF683231F45A2FD8DF683292
:107BD00011F4882708958FE05F915F91CACFE7DFA6
:107BE000CCDF603169F4572F550F5E70516AC7DFE3
:107BF000603431F4CDDF683519F411968827B9CF98
:107C00008FE0B7CF052ED3DF502DB9DF683219F4DE
:107C100011968827AECF8FE00895AFDF6830A9F4C2
:107C2000572F5770550F5169AADF603471F4ABDFDD
:107C3000603559F4A52FACDF683539F4BB27550FF3
:107C4000AA1F08F4B095882794CF8FE092CF882799
:107C5000D83020F082E24F914F914FEF0895F7DF37
:107C6000F999FECFD2BDC1BDF89A40B521960895CD
:107C7000EEDF8827F999FDCFD2BDC1BDF89A40B497
:107C8000441611F42196089540BDF894FA9AF99A91
:107C90007894F999FECFF89A21960895AF93DFDF93
:107CA0004193AA95E1F7AF910895AF934191E0DF39
:107CB000AA95E1F7AF9108954EBD4DB547FFFDCFB1
:107CC0004EB5089588272C9847EDF6DF4427F4DF5A
:107CD0002C9A4C7B4432B1F34C31A1F38827443ABF
:107CE00019F04C3909F081E108958827EBDF8030E5
:107CF00021F040E040939C1008954C3911F448E085
:107D0000F9CF40E1F7CFF1DF403009F40895440F97
:107D1000440F440F440F4A950895AA0FBB1F4B2FE1
:107D2000CBDF4A2FC9DF422DC7DFB695A79508954F
:107D3000803059F44F93C6DF803031F42C9845E5FC
:107D4000BBDFEBDF2C9ABEDF4F910895803059F4F2
:107D50004F93B8DF803031F42C9843E5ADDFDDDFA1
:107D60002C9AB0DF4F910895803051F44F93AADFE1
:107D7000803029F42C9846E89FDFCFDF2C9A4F9172
:107D800008951196B0939D10A0939E101197ECCF7B
:107D90002DD2CEDF48D0E8CF7F93772710D07F91C8
:107DA00008957F9371E00BD0D42F72E008D0C42FD8
:107DB0007F9108957F9373E002D07F910895803082
:107DC00099F480DF803081F42C9842ED75DFAA0FA2
:107DD000BB1FA3954B2F70DF4A2F6EDF472F6CDF41
:107DE000B695A79502D02C9A089566DF65DF64DF0B
:107DF00063DF62CF8030B1F465DF803099F42C9876
:107E000042ED5ADFAA0FBB1F4B2F56DF4A2F54DF1C
:107E1000472F440F51DFB695A795E7DFD42F4CDFEE
:107E2000C42F2C9A08957F9370E010D07F9108950D
:107E30007F9371E04D2F0AD072E04C2FC0DF7F910D
:107E400008957F9373E0BBDF7F9108958030A1F4A4
:107E50004F9338DF4F91803079F42C984F9347E857
:107E60002BDF442729DF41E027DF472F25DF4F9114
:107E70004F9322DF2C9A4F910895803091F422DFA6
:107E80008030D1F72C984F9347E816DF442714DF52
:107E900040E012DF472F10DF4F914F930DDF2C9AF8
:107EA0004F9108958030D1F4DF93CF934F935F9338
:107EB00009DF803079F42C9847E8FEDE4427FCDEA9
:107EC0004427FADE40E0F8DE55274991F5DE5A9561
:107ED000E1F72C9A5F914F91CF91DF910895803017
:107EE000B1F44F935F93EEDE803079F42C9847E83D
:107EF000E3DE4427E1DE4427DFDE40E0DDDE552718
:107F00004FEFDADE5A95E1F72C9A5F914F91089581
:107F10008030E1F4DF93CF934F935F93D3DE8030D3
:107F200089F42C9846EDC8DE4427C6DE4427C4DE1B
:107F300040E0C2DE4427C0DE5527BEDE49935A9595
:107F4000E1F72C9A5F914F91CF91DF910895BF9304
:107F5000AF93DF93CF934F935F937F93C6DE403011
:107F600001F4BDDF4FE05FDF44276BDFAA27BB27AB
:107F7000FBDE11964DEFCA2FCF70C13009F44CEFE4
:107F800052DF44275EDFCC27DD2752DFEDDE11967E
:107F9000A03019F445EE0E94BC3240919C10B417F9
:107FA00049F70AC0BF93AF93DF93CF934F935F938B
:107FB0007F939BDE403091F47F915F914F91CF9101
:107FC000DF91AF91BF910895B42FAA271197F2DEE8
:107FD000C42FBB27AA27EEDE4C1731F4A9DEEADE58
:107FE00043952FDFC1DEE8CF1196E4DE4C17E1F7B1
:107FF000F5CFDF93CF934F939BDE4DEFCA2FCF701A
:10800000C13009F44CEF0FDFCCDE219611DF67DFC2
:10801000ABDE4F91CF91DF910895FF93EF93DF9304
:10802000CF93BF93AF93AA27BB27ED015EDE40300D
:10803000A1F0F42FB1DE4C3F41F04D3F31F04B3A0F
:1080400021F04F3018F0403908F421961196BF17EF
:1080500089F74427DF1709F441E06FC00F93BF93FE
:10806000AF934F93AA27BB27ED01FD013EDE4030C1
:1080700099F0042F91DE4D3F49F4DF93CF9391DEC9
:108080004D2FCF91DF914F3F21F021964C3F09F4C6
:1080900031961196B01771F74F91AF91BF910F9133
:1080A0000895FF93EF93DF93CF934F932F931DDEAC
:1080B0004030A9F0AA27BB276FDE242FB0919D1076
:1080C000A0919E1040911401B41710F0A2E0BB27BC
:1080D000FD0162DE4D3F31F464DED21718F42F91BA
:1080E0004F912DC0159640919C10B41709F4BB27F1
:1080F000BF1779F7AE1769F7AA27BB2719DE4CDE41
:108100004F3F31F0405F242F8EDE2EDEDF01E1CFC6
:10811000AFEFBFEFE4CFFF93EF93DF93CF93BF9326
:10812000AF934F935F936F937F93DFDD403061F4A4
:1081300081E17F916F915F914F91AF91BF91CF910D
:10814000DF91EF91FF91089551D0B41710F08BE1BA
:10815000F0CF22DE4C3F11F087E1EBCF40917A0166
:10816000403011F48BE1E5CF413810F08BE1E1CFE5
:1081700075DFD03021F4C41710F488E1DACFCCE3F6
:10818000DFE050E06FEF69935A95E9F7A8DE1196AA
:10819000B0939D10A0939E1040917A01CCE3DFE054
:1081A0004F937FDFB993A9934BEA3DDEDF93CF93E3
:1081B000F8DD21963DDECF91DF91FCDD42DEE1DD91
:1081C000F1DE4F914A9561F711D0CCE3DFE06ADE32
:1081D00040917C0128DEDF93CF93E3DD219628DEFA
:1081E000CF91DF91E7DD2DDEBFDDA3CFA091780138
:1081F000A295BA2FA07FBF70119608950E94240106
:108200004F935F937F937727F1DFC6DD4C3F69F093
:10821000F1DDDF3F49F0BF93AF93DE01EADEAF91BE
:10822000BF91C0DE7F5FA1F7E4DE7F915F914F9148
:108230000C941D010E9424014F935F937F932F9311
:10824000AA27BB273FDDA8DD242FD0DFA5DD4C3FCB
:1082500039F489E12F917F915F914F910C941D0129
:1082600070917A01703810F08BE1F4CFC3DDDF3FFD
:1082700011F48BE1EFCFDE01CCE3DDE040917C0136
:10828000413009F4D395423009F4DE5F0BDEDF9311
:10829000CF9387DDD21759F02196CADDCF91DF91B8
:1082A0007BDDC1DD87DDCDDD5FDD7CDED3CFA1DE13
:1082B000F8DE77DD2196BCDDCF91DF914BEAB3DDAF
:1082C00079DDBFDD51DDED0191DF32DD70917A01A5
:1082D000770F4D2FD2DD73954C2FCFDD5DDDA3DD04
:1082E00069DDAFDD41DDB6CF0E9424014F935F937E
:1082F0007F937CDF51DD4C3F31F48EE17F915F91C4
:108300004F910C941D0170917A01703810F08BE13F
:10831000F5CF70DDDF3F11F48BE1F0CFDE0108DD3A
:10832000CCE3DDE040917C01413009F4D39542304B
:1083300009F4DE5FEDDDE2CF0E9424014F935F93ED
:108340007F9354DF29DD4C3F11F48EE1D7CF77279F
:1083500051DDDE0170E0E8E8F1E04CDDD193C1933E
:1083600073957032D1F7CACF0004080D11161A1F89
:1083700023282C3035393D42464A4F53575B5F64C2
:10838000686C7074787C7F83878B8F92969A9DA19E
:10839000A4A7ABAEB1B5B8BBBEC1C4C6C9CCCFD122
:1083A000D4D6D9DBDDDFE2E4E6E8E9EBEDEEF0F28E
:1083B000F3F4F6F7F8F9FAFBFCFCFDFEFEFFFFFF15
:1083C000FFFFFFFF000000CCC000333000FFF000D3
:1083D000000CCCCCCCCC333CCCFFFCCC000333CC5D
:1083E000C333333333FFF333000FFFCCCFFF333FBF
:1083F000FFFFFFFFA5A5A506FF600000000000002D
:10840000000000000000000000000000000000006C
:1084100000000000000000000EAE000004E000AA12
:10842000E800EE4E000000444040AA000066FF66EF
:108430006842C4A248A000000044000048884042AE
:1084400022400A4A0004E40000048000E00000002A
:1084500040224880EAAAE04C44E0E2E8E0E2E2E0C0
:10846000AAE220E8E2E0E8EAE0E24880EAEAE0EABC
:10847000E2E00404000404802484200E0E0084241E
:1084800080C268E400EEE04AAEA0CACAC068886054
:10849000CAAAC0E8C8E0E8C88068EA60AAEAA0E41E
:1084A00044E0E22A60AC8CA08888E0AEAAA0CAAA08
:1084B000A04AAA40EAE8804AAA60EAECA068E2C0C2
:1084C000E44440AAAAE0AAAA40AAAEA0AA4AA0AA46
:1084D0004440E248E064446004A400C444C04A004C
:1084E000000000E04400004AAEA0CACAC06888602C
:1084F000CAAAC0E8C8E0E8C88068EA60AAEAA0E4BE
:1085000044E0E22A60AC8CA08888E0AEAAA0CAAAA7
:10851000A04AAA40EAE8804AAA60EAECA068E2C061
:10852000E44440AAAAE0AAAA40AAAEA0AA4AA0AAE5
:108530004440E248E024C4204444448464808842A7
:04854000208CEC801F
:1086000000F900F5F3F1F2FC00FAF8F6F4EB5E0085
:10861000F7000000007131000000797361773200CB
:108620000063786465343300002076667472350028
:10863000006E6268677A360000006D6A7537380030
:10864000002C6B696F303900002E2D6C00707E009D
:1086500000000000002700000000EA2B00230000BB
:10866000003C00000000EC00003100343700000046
:10867000302C32353638ED00FB2B332D2A390000F3
:1086800000F900F5F3F1F2FC00FAF8F6F4EB000063
:10869000F70000000051210000005953415722000B
:1086A00000435844452440000020564654522500BB
:1086B000004E4248475A260000004D4A552F2800D8
:1086C000003B4B494F3D2900003A5F4C00503F00B2
:1086D00000000000006000000000EA2A00270000FF
:1086E000003E00000000EC000031003437000000C4
:1086F00030E932353638ED00FB2B332D2A390000B6
:108700000000000000000000000000000000000069
:108710000000000000000000000000000000000059
:108720000000000000000000000000000000000049
:1087300000000000000000C000000000000000C1B8
:10874000000000000000000000002F0000000000FA
:1087500000000000000000000000EA000000C2006D
:10876000000000000000000000E100E2E000000066
:10877000E8E9E500E3E4ED00FB2BE72D2AE6000045
:1087800000000000000000000000000000000000E9
:108790000000000000400000000000000000000099
:1087A00000000000000000000000000000000000C9
:1087B000000000000000000000000000007B5B00E3
:1087C00000000000007D5D000000000000007E0051
:1087D00000000000000000000000005C000000003D
:1087E000007C00000000000000E100E2E00000006A
:1087F000EFEEE500E3E4ED00FB2BE72D2AE60000B9
:1088000000F900F5F3F1F2FC00FAF8F6F4EB5E0083
:10881000F70000000071310000007A7361773200C8
:108820000063786465343300002076667472350026
:10883000006E62686779360000006D6A753738002F
:10884000002C6B696F303900002E2F6C3B702D00AF
:10885000000027005B3D00000000EA5D007E000094
:10886000000000000000EC00003100343700000080
:10887000302C32353638ED00FB2B332D2A390000F1
:1088800000F900F5F3F1F2FC00FAF8F6F4EB000061
:10889000F70000000051210000005A5341574000EA
:1088A00000435844452423000020564654522500D6
:1088B000004E424847595E0000004D4A55262A00A6
:1088C000003C4B494F292800003E3F4C3A505F0086
:1088D000000022007B2B00000000EA7D007C0000ED
:1088E000000000000000EC00003100343700000000
:1088F00030E932353638ED00FB2B332D2A390000B4
:108900000000000000000000000000000000000067
:108910000000000000000000000000000000000057
:108920000000000000000000000000000000000047
:1089300000000000000000C000000000000000C1B6
:10894000000000000000000000002F0000000000F8
:1089500000000000000000000000EA000000C2006B
:10896000000000000000000000E100E2E000000064
:10897000E8E9E500E3E4ED00FB2BE72D2AE6000043
:1089800000000000000000000000000000000000E7
:1089900000000000000000000000000000000000D7
:1089A00000000000000000000000000000000000C7
:1089B00000000000000000000000000000000000B7
:1089C00000000000000000000000000000000000A7
:1089D0000000000000000000000000000000000097
:1089E000000000000000000000E100E2E0000000E4
:1089F000EFEEE500E3E4ED00FB2BE72D2AE60000B7
:108A0000FFFFFFFFFFFFFFFFFFFFFFFEFEFEFEFE7B
:108A1000FEFEFDFDFDFDFDFCFCFCFCFBFBFBFBFA93
:108A2000FAFAF9F9F9F8F8F8F7F7F7F6F6F5F5F4D0
:108A3000F4F3F3F3F2F2F1F1F0EFEFEEEEEDEDEC33
:108A4000EBEBEAEAE9E8E8E7E6E6E5E4E4E3E2E1BD
:108A5000E1E0DFDEDEDDDCDBDADAD9D8D7D6D5D56A
:108A6000D4D3D2D1D0CFCECDCCCBCBCAC9C8C7C638
:108A7000C5C4C3C2C1C0BFBEBCBBBAB9B8B7B6B526
:108A8000B4B3B2B0AFAEADACABA9A8A7A6A5A4A233
:108A9000A1A09F9D9C9B9A989796959392918F8E5B
:108AA0008D8C8A89888685848281807E7D7B7A7997
:108AB0007776747372706F6D6C6B696866656362EC
:108AC000615F5E5C5B595856555352504F4D4C4A4E
:108AD000494746444341403E3D3B3A3837353332BF
:108AE000302F2D2C2A2927262422211F1E1C1B193A
:108AF0001816141311100E0D0B09080605030200B9
:108B00000C11161A1E2225282B2D2F313233333407
:108B100034343434343434343535363738393B3CF6
:108B20003E40434547494B4D4F5152535454545482
:108B3000545351504E4C4A4745423F3D3A383634E3
:108B40003231302F2E2E2E2F303132333536383A07
:108B50003C3E4042444647494A4B4D4E4E4F505092
:108B60005050505050504F4E4D4C4B494846434149
:108B70003E3B37332F2B27221D18130D0802FDF81B
:108B8000F3EEE9E5E1DDDAD7D4D2D0CECDCCCCCB53
:108B9000CBCBCBCBCBCBCBCBCACAC9C8C7C6C4C344
:108BA000C1BFBCBAB8B6B4B2B0AEADACABABABAB98
:108BB000ABACAEAFB1B3B5B8BABDC0C2C5C7C9CB17
:108BC000CDCECFD0D1D1D1D0CFCECDCCCAC9C7C5D3
:108BD000C3C1BFBDBBB9B8B6B5B4B2B1B1B0AFAF28
:108BE000AFAFAFAFAFAFB0B1B2B3B4B6B7B9BCBE51
:108BF000C1C4C8CCD0D4D8DDE2E7ECF2F7FD02075F
:108C0000000A141D272F383F464B505457595959C5
:108C1000585654504C48433E39332E2925201C19B0
:108C200016141211111112131517191C1F222527C2
:108C30002A2C2E303132323232312F2D2B28252260
:108C40001F1C191613110F0D0C0B0A0A0A0B0C0E20
:108C500010121416181A1C1E1F2020201F1E1C196B
:108C600016120D0803FDF7F0EAE3DDD6D1CBC6C23C
:108C7000BFBDBBBABBBCBEC2C6CBD1D7DFE6EFF728
:108C80000008101920282E34393D41434445444200
:108C9000403D39342E29221C150F0802FCF7F2ED55
:108CA000E9E6E3E1E0DFDFDFE0E1E3E5E7E9EBED83
:108CB000EFF1F3F4F5F5F5F4F3F2F0EEECE9E6E3B9
:108CC000E0DDDAD7D4D2D0CECDCDCDCDCECFD1D37D
:108CD000D5D8DADDE0E3E6E8EAECEDEEEEEEEDEB3A
:108CE000E9E6E3DFDAD6D1CCC6C1BCB7B3AFABA9F6
:108CF000A7A6A6A6A8ABAFB4B9C0C7D0D8E2EBF57B
:108D000080675342352B221C16120E0C09070605EC
:108D1000040000000000000000000000000000004F
:108D2000807E7B79777572706E6C6A686664636149
:108D30005F5D5C5A5857555352504F4D4C4B494804
:108D40004745444341403F3E3D3C3B39383736354B
:108D50003433323231302F2E2D2C2B2B2A29282838
:108D60002726252524232322222120201F1F1E1DE4
:108D70001D1C1C1B1B1A1A19191818181717160076
:108D8000890091009A00A300AD00B700C200CE0098
:108D9000DA00E700F4000301120123013401460167
:108DA0005A016E0184019B01B301CD01E901060264
:108DB0002502450268028C02B302DC020803360376
:108DC00067039B03D2030C0449048B04D0041905E8
:108DD0006705B90510066C06CE063507A307170808
:108DE000930815099F09320ACD0A720B200CD80C82
:108DF0009C0D6B0E460F2F1025112A123F13641481
:108E0000F894A0E02A2EA1E03A2EA0E1AEBFAFEF89
:108E1000ADBFB0E0A0E0AA95F1F7BA95D9F7AAEBFB
:108E2000A4B9AFEFA5B9A0E8A7B9A0E0A8B9A0EF91
:108E3000AAB9AFEFABB9A6B1AF71A09335014B9909
:108E40005DC0B2ECB0938000B9E1B0938100F4E072
:108E5000A2FFF4E0F0938700FEEFA2FFF6EFF0939D
:108E6000860020928900FAE5F0938800A2E0A093A2
:108E70006F00A0E4A4BDA1E0A5BDA1E3A7BD209221
:108E8000C000A0E1A093C100A6E6A093C200E0EA62
:108E9000FFE87ED0A2E2B591B993AA95E1F705B7B4
:108EA000036005BF0E7F05BF7894A8EC68D0B09131
:108EB000C600B83719F0AA95C9F720C0E0ECFFE862
:108EC00067D045E140D0C8EDD1E020D046E03BD0AE
:108ED000E0E0F0E0CCE3DFE019D046E034D0CCEBCA
:108EE000DFE014D0FE3820F40E946779329678943F
:108EF00046E029D0AEEEB1E01BD0ECCFF89405B738
:108F0000016005BF0C7F05BF0C94000028D04430E1
:108F100039F446E018D0B0913101B030E1F7EECF2E
:108F200050E81DD01CD01BD049935A95E1F717C0CB
:108F30004F2F429501D04F2F4F70405D4A3308F0BC
:108F4000495F4D930895BF93B0913101B030E1F77F
:108F500040933201BA95B0933101BF910895BF9308
:108F6000B0913301B030E1F7BA95B0933301B091CD
:108F70003301B030E1F740913401BF910895AF93D0
:108F8000A82DA73EE9F3A82DA73EE9F7AF910895D4
:108F9000C8EDD1E0A2E2B591B993AA95E1F70895A1
:108FA0004156522D436869704261736963322028CB
:108FB0004631313D557064617465205379732920C1
:108FC000426F6F746C6F61646572204572726F726C
:108FD000202845534320746F206578697429202028
:0E900000202020202020202020202020FFFFE4
:0E9C0000202020202020202020202020FFFFD8
:0EA80000202020202020202020202020FFFFCC
:0EB40000202020202020202020202020FFFFC0
:0EC00000202020202020202020202020FFFFB4
:0ECC0000202020202020202020202020FFFFA8
:0ED80000202020202020202020202020FFFF9C
:0EE4000048656C6C6F20576F726C64204EFF85
:10E410000E94670000EC0E9456000E9473000000FA
:10E4200048656C6C6F20576F726C642100000EE0C1
:10E430000E9456000E947300020070726573732080
:0CE4400071000E947B004137E1F7089555
:10F000000C94004700000000000000000000000019
:10F0100000000000000000000000000000000000F0
:10F0200000000000000000000000000000000000E0
:10F03000000000000C941C784F935F936F93FF9334
:10F04000EF93DF93CF93BF93AF930F921F92FFB7CE
:10F05000FF93C4E1D1E0B9A5B7FF5C98B7FD5C9A16
:10F060004B99BE7F4B9BB160B9A7830C921CE9A161
:10F07000F92DF03029F4F82DFA3010F1F63EF8F0C1
:10F08000FCE0E2FFFDEE8F1639F45E98E3FF17C057
:10F09000B2E8B093800013C0F1E1E2FFF3EF8F1606
:10F0A00039F45E9AE3FF0BC0B2ECB093800007C066
:10F0B000F9E3E2FFF7E08F1611F4882499242CC0BD
:10F0C000A0918400A63EE0F3A73E00F0A83E00F029
:10F0D000A93E00F0AA3E00F0A8EDB1E0F6EFF80D71
:10F0E000C0E2ED91549140E060E848B9ED9156FDE1
:10F0F00066B90000000055FD66B9049054FD66B97C
:10F10000CA95000053FD66B90000000052FD66B9C3
:10F11000502D59F7000028B814D0E091C600E6370A
:10F1200011F40C947E47FF91FFBF1F900F90AF9199
:10F13000BF91CF91DF91EF91FF916F915F914F91CF
:10F140001895A0913D01E0913301E03091F0EF3F3F
:10F1500021F4A0FD0EC0EEE30CC0EA95F5EFB491EA
:10F16000B5FF07C0B0913401B695A0FBB7F9B093D5
:10F170003401E0933301E0913101E03091F0EF3F51
:10F1800019F4E0E5AF770DC0EA95F5EFB491B4FF5F
:10F1900008C0B0913201B0FB0894B795A7F9B093BD
:10F1A0003201E0933101A0933D010895A0913D010A
:10F1B000E0913301E03091F0EF3F21F4A0FD0EC06B
:10F1C000ECE70CC0EA95F5EFB491B7FF07C0B0913A
:10F1D0003401B695A0FBB7F9B0933401E093330145
:10F1E000E0913101E030E9F2EF3F19F4E0E9AF7767
:10F1F000D8CFEA95F5EFB491B6FFD3CFB0913201F5
:10F20000B0FB0894B795A7F9B0933201CACF4091EB
:10F210001801C8EFD7E00E94383E409165010E9476
:10F22000383E0895C8EFD7E00E942F3E4093180162
:10F230000E942F3E409365010895FF93EF93DF9363
:10F24000CF93AF93F5D0E0934001F0934101AF919C
:10F25000CF91DF91EF91FF910895E0914001F091FE
:10F260004101A0E2A99FE00DF11DB096C0EBD1E0F5
:10F27000A0E2B591B993AA95E1F7BFEFB9930895CC
:10F2800047B740FDFDCFB7BFE89547B740FDFDCF7D
:10F29000089547B746FF0895B1E1F2DFFACFF89439
:10F2A0004E2F407E19F4B3E0EBDFF3DFA0E10990CD
:10F2B0001990B1E0E5DF3296AA95C9F7E03009F080
:10F2C00008953297B5E0DCDFE4DF32960895F894D4
:10F2D0004F93BF93AF93B3E0D3DFDBDF3297CCE341
:10F2E000DFE0A0E8329609901990B1E0C9DFAA9555
:10F2F000C9F7B5E0C5DFCDDFAF91BF914F9108955C
:10F30000E0914001F0914101B097ACE0B591B99323
:10F31000AA95E1F7A0913501A7FD0895A6EAB2E00C
:10F32000CA0FDB1FACE0B0913801B993AA95E9F799
:10F330000895E0E0F0E9A0E0BCE0492F403029F377
:10F34000EA0FFB1F4A95FACF409149014770AF93EE
:10F35000ECE0F0E9ACE0A49FF00D4491EC50AF91EB
:10F360000895F89463D0C0EBD1E0A3EEB1E05CE087
:10F370004D9149935A95E1F742E4499353E140E2B4
:10F38000B9935A95E9F7A0978ADF9927B3E2B99F15
:10F39000A4E4B2E0A00DB11DC8E8D1E050E24D9167
:10F3A00049935A95E1F7299250E24A91403219F473
:10F3B00028825A95D1F70E94471AC0EBD1E06FDF3F
:10F3C00093959F3519F77894089530D0A3EEB1E066
:10F3D0005CE045914D935A95E1F77496992750E278
:10F3E000A0EBB1E045914D935A95E1F7A8E8B1E063
:10F3F00040E253E24D935A95E9F7FF93EF939F93C1
:10F400000E94281B9F91EF91FF91C8E8D1E0B3E2E1
:10F41000B99FA1E4B2E0A00DB11D53E249914D9313
:10F420005A95E1F793959F35D1F60895409149019A
:10F43000AF93BF93E0E0F0E947704295A0ECA49F42
:10F44000E00DF11DBF91AF910895CCE3DFE04CE0FA
:10F4500050E259934A95E9F75FEF599343E150E23F
:10F4600059934A95E9F740EF5FEF59934A95E9F7C9
:10F47000DDDF2DDF3296CCE3DFE040E25FEF599332
:10F480004A95E9F74BE04F9322DF32964F914A9528
:10F49000D1F778940895472F4770CADFFF93EF9311
:10F4A000C5DFAF91BF914CE04F93CCE3DFE040E08C
:10F4B000559159934A95E1F7FF93EF93FD0107DFCB
:10F4C0003296DF01EF91FF914F914A9569F7789459
:02F4D00008959D
:10F50000010101010101210101010101012181012B
:10F510000100002100110101010121D101010101BE
:10F520002101110101010121D1010101012101117B
:10F530000101010121D101010101010111010101BB
:10F540000101D1010101010101110101010101C10B
:10F55000010101010101010101000101C1010101DC
:10F56000010101010101010001C1010101010100CD
:10F57000010101010101410001010101010101003D
:10F58000000000400000000000000000000000003B
:10F59000000000000000000000000000000000006B
:10F5A000000000000000000000000000000000005B
:10F5B000000000000000000000000000000000004B
:10F5C000000000000000000000000000000000003B
:10F5D000000000000000000000000000000000002B
:10F5E000100000000000000000000000000000000B
:10F5F00020000000000000000000000000000000EB
:10F60000009010800090108000901080009010807A
:10F61000FC28288004C0145028282800000000007E
:10F6200000000000000000000000000000000000DA
:10F6300000000000000000000000000000000000CA
:10F6400000000000000000000000000000000000BA
:10F6500000000000000000000000000000000000AA
:10F66000000000000000000000000000000000009A
:10F67000000000000000000000000000000000008A
:10F6800028C004C00000000000000000000000804E
:10F69000C0A0888400000000000000002088FCB4A6
:10F6A0000028000008A08080000004C028800024FA
:10F6B00028008000000044288000C004C418000016
:10F6C00000282828280028281818280000000000F2
:10F6D0008090808008A084408080C8A400004C8472
:10F6E00000000000000000008080601800802828D2
:10F6F000280000002828002828282800002CE8904E
:10F700000090108000901080009010800090108079
:10F710007C444480A8A814504844440024000000BD
:10F7200000183C3C185028280C3000000000000055
:10F73000241824400C401440242400000C003024E1
:10F7400024244424444040246424106460646424D9
:10F7500044244424406464646464404800481800BD
:10F76000300060000400140060180C6028000000E5
:10F7700000000000300000000000000C18306000A5
:10F7800028A004C0808044283C3C3C000044A88061
:10F79000C0A08884000000000000008040847C58E5
:10F7A000182800001090808004C004C028FC287C29
:10F7B00028440C00000044EC8000C004C424000075
:10F7C00000282828286C2828C01828640000000079
:10F7D0008088A41010908440C004C8A400008C80CD
:10F7E000287C008080004084FCF8303000002448F1
:10F7F000280000002828002828282800002CE8C01D
:10F800000090108000901080009010800090108078
:10F81000FC44448080801450444444283C00000050
:10F8200000183C3C20546C181818181800000004EC
:10F830006428640C14603064646428281800186418
:10F84000646464646460606464180C6C605864642C
:10F8500064646464186464646464046000183C0054
:10F860001800600004003400600000601800000010
:10F870000000000030000000000000181818601898
:10F88000449008A0C4C4806C0000001C1844A880E8
:10F89000C0A0888400000000000080804084FCB488
:10F8A0002428282820888080A4A00C60448044401C
:10F8B00028440C40844444800000C0046C2400446C
:10F8C00000282828286C8080C018445440844810A0
:10F8D0008084BCB020888820D834C8A440848C8020
:10F8E0002C7C00C4C4448080C0082830008020885C
:10F8F000280000002828002828282800002CE8A03C
:10F900000090108000901080009010800090108077
:10F910007C808080808010908480804424186424BF
:10F9200000183C40780C7830300C7C180000000C3B
:10F93000681804183C44600C6464282830400C04A7
:10F94000046464606460606064180C78607C546473
:10F9500064646460186464643C640C60301864001F
:10F960000C2444242C2430207428146C185C742437
:10F970004824742448646464646440181818300C83
:10F9800044881090C4BC446C24246434286C6C807B
:10F99000C0A08884000000000080808080807CEC13
:10F9A000404444442088408490A00C6044FC286477
:10F9B00080440C40844444280000C0046C2400802F
:10F9C00028444444446C80806018C44C600C18186F
:10F9D0008080BC1040848820E82CC8A480804C849F
:10F9E000EC2400C4EC448080C008144800802088C7
:10F9F000280000002828002828282800002CE8E4F7
:10FA00000090108000901080009010800090108076
:10FA1000FC808080B098109080ECEC44003C6464E2
:10FA20000018003C24183000300C2440004000181E
:10FA30007C180C0C6C044418242000006000040C9A
:10FA40002C6444606444447040180C50607C7C64B6
:10FA50004464442418646464183C18607C180000F2
:10FA6000000464606864486454180C78187C54641A
:10FA70006C6C5460306464643C640C30180C188006
:10FA800080841090C4F8806C04646440406C6C8086
:10FA9000C0A0888400000000808080808080FCB44A
:10FAA0001880442840844084808418308080282432
:10FAB00000440C40844444440000C00428241880BE
:10FAC0008080844080A800006018C480A008402482
:10FAD000A4B0BC4080808080E82CC8A488104084FA
:10FAE000E42428C4EC44D480C00814848080208896
:10FAF000288020882088808020888020882CE8F03A
:10FB00000000000090909090101010108080808075
:10FB10007C8080801090B098408080440040646475
:10FB2000001800401C307800300C7C182800003091
:10FB300054181804400464186404282830400C1831
:10FB40007C4064606460606464180C78606468641D
:10FB5000607C780418643C7C3C1830600C18000011
:10FB6000002064606440306464180C50187C646445
:10FB70006C6C602430646464182C181818180C0C11
:10FB800080842088C4C444C420646430286C6C80A1
:10FB9000C0A08884000000008080808080807CEC91
:10FBA00018008044408440848080301880FC801895
:10FBB00044448040844444440000C0042800244459
:10FBC0008080844080A800443018C480A00824406D
:10FBD000BCD0A41084404084E82CC8A44C8480800D
:10FBE000482428C4EC44F880C0081484808020880D
:10FBF000288020882088808020888020882CE82801
:10FC00000000000090909090101010108080808074
:10FC1000FC8080801090808084C4A8440000643CF4
:10FC20000000003C44686C00181818181800286080
:10FC3000641830640C646430640C281818001800D0
:10FC40007C6464646460606464186C6C60646464A4
:10FC500060686C6418643C7C641860600018000084
:10FC6000006464646460302064180C781864646410
:10FC7000482460043C683C7C3C0830181818041880
:10FC800044882088C4C4808064646818186C6C80C0
:10FC9000C0A0888400000080808080808080FCB4C8
:10FCA000400080804084208880843018DC80284098
:10FCB00000446040844444280000C0046C0024C414
:10FCC00044444444446C80443018C44C600C1818BC
:10FCD000BCB0808084402088E44CC4C44C848080C4
:10FCE000282400C4EC44D4D0FCF8148480002828D4
:10FCF000280028280000280028282820882CE83000
:10FD00000000000090909090101010108080808073
:10FD10007C4480441450808044EC442800004458C3
:10FD20000018003C18082C000C300000300028009F
:10FD3000242440240C242430242800300C003018C3
:10FD4000246444244440602464242864406464247B
:10FD5000602C64241824182464184048004800408B
:10FD6000002044242424300464246C6C246464241F
:10FD7000600C6044182C183C6404400C18300400DB
:10FD8000449040848080442820242C0000A8448093
:10FD9000C0A08884000080808080808040847C585F
:10FDA000240080288080208890A0600CDCFC44180F
:10FDB00028446040844444EC0000C0046C002400EB
:10FDC00028002828286C804418184454408410487F
:10FDD000BCB0808080801090D094C0048C8040841F
:10FDE000284000C4C444FCF880802884800028286F
:10FDF000280028280000280028282820882CE830FF
:10FE00000000000090909090101010108080808072
:10FE1000FC4480441450A8A84080440000006000C6
:10FE200000000000000000000000000000000000D2
:10FE300000000000000000000000000000000000C2
:10FE400000000000000000000000000000000000B2
:10FE500000000000000000000000000000000000A2
:10FE60000000000000000024000028000000000046
:10FE700060080000000000000024000000000000F6
:10FE800028A08080000000000000000000A844803E
:10FE9000C0A0888400808080808080804084FCECCA
:10FEA0001800444480801090A4A0C004DC806C3C06
:10FEB00000446000004400800080C004C4002400AE
:10FEC00028002828286C282818182864000000001A
:10FED000A4B08080844008A0C8A480808C800000EA
:10FEE000444000808000D4F8408430480000282836
:10FEF000280028280000280028282824482CE8006A
:10FF00000000000090909090101010108080808071
:10FF10007C2880281450109080EC28000000C0003D
:10FF200000000000000000000000000000000000D1
:10FF300000000000000000000000000000000000C1
:10FF400000000000000000000000000000000000B1
:10FF500000000000000000000000000000000000A1
:10FF60000000000000000000000000000000000091
:10FF70000000000000000000000000000000000081
:10FF800028C0808000000000000000000000008009
:10FF9000C0A08884808080808080808020887C5879
:10FFA00000004480808008A004C0C0048CFCA858D5
:10FFB00000006000004400280080C004C40000006D
:10FFC00028002828280028281818280000000000E9
:10FFD0008080000084400000C8A400004824000085
:10FFE00000000000000080800000600080002828E1
:10FFF000280028280000280028282828282CE80085
:00000001FF
